:100000000C941E060C9430280C945D280C94460623
:100010000C9446060C9446060C9446060C94460630
:100020000C9446060C9446060C94EF120C9446066B
:100030000C9446060C9446060C9446060C94460610
:100040000C948A280C9446060C94782C0C94BB2CA7
:100050000C9446060C9446060C9446060C944606F0
:100060000C9446060C9446069E180019DF18E218F8
:10007000E518E818EB18EE18F1180019FA18321AFA
:10008000341A341A321A341A341A341A341A341A02
:10009000341A341A341A341A341A341A341A341AF0
:1000A000B819341A341A341A341A341A2919341A69
:1000B000341A341A341A341A341A341A341A341AD0
:1000C000341A341A341A341A341A341AC419C419A2
:1000D000C419C419C419C419C419C419C419341AC7
:1000E000341A341A341A341A341A2919C319C31990
:1000F000C319C319341AD119D719DD19E319E9192C
:10010000EF19F519FB19051A0F1A191A231A6A198A
:100110002C19341A341A341A341AB819341A341AF5
:10012000341A341A341A341A341A341AC219C21945
:10013000C219C219341AD119D719DD19E319E919ED
:10014000EF19F519FB19051A0F1A191A231A6A194A
:100150002C19341A341A341A341AB819671A671A4F
:10016000671A671A671A671A671A671A671A671A87
:10017000671A671A671A7D1B7D1B7D1B7D1B7D1B04
:100180007D1BAC1AB61AC01ACA1A271B311B401B9A
:10019000511BD91CEE1CFA1C031D121D371D401DDE
:1001A000891D521D9E20A420AA20B120BF20E1203D
:1001B000FF20456E746572206D656E752E2E2E00C3
:1001C000546F67676C6564206D6963726F50504D42
:1001D00000546F67676C656420696E76657274653C
:1001E000642050504D2100546F67676C6564205443
:1001F00058206D7574696E672100546F67676C6570
:10020000642074656C656D65747279210050726F3D
:10021000746F636F6C206572726F72207769746897
:100220002052580054696D656F7574207768656E4B
:1002300020636F6E6E656374696E6720746F205201
:100240005800507265737320616E79206B65792058
:10025000746F2063616E63656C00436F6E6E6563DF
:1002600074696E6720746F2052582C20706F776508
:100270007220757020746865205258202877697440
:10028000682062696E6420706C7567206966206EF4
:100290006F74207573696E6720616C776179732064
:1002A00062696E642900546F67676C656420276912
:1002B0006D6D656469617465206F75747075742700
:1002C00000546F67676C65642027736C61766520E6
:1002D0006D6F64652700546F67676C6564202761E4
:1002E0006C776179732062696E642700546F676769
:1002F0006C65642050504D206368616E6E656C20A3
:100300006C696D69740053657420525353492069B8
:100310006E6A656374696F6E206368616E6E656C8A
:100320002028303D3D64697361626C652900536526
:10033000742050504D206D696E696D756D20737914
:100340006E630053657420626561636F6E20696E31
:1003500074657276616C0053657420626561636FC9
:100360006E2064656C617900536574206265616319
:100370006F6E206672657175656E637920696E2097
:10038000487A3A20303D64697361626C652C205074
:10039000783D504D52206368616E6E656C20782CFC
:1003A0002046783D465253206368616E6E656C202E
:1003B00078005365742050574D2073746F7020641B
:1003C000656C61792028302064697361626C6564B2
:1003D0002C20312D323535203D3D20302E317320FB
:1003E0002D2035306D696E29005365742050504DB5
:1003F0002073746F702064656C61792028302064EC
:10040000697361626C65642C20312D323535203D75
:100410003D20302E3173202D2035306D696E29003E
:10042000536574206661696C736166652064656CF0
:1004300061792028302064697361626C65642C20C6
:10044000312D323535203D3D20302E3173202D2089
:1004500035306D696E29002A2A2A2A2A2A2A2A2A50
:100460002A2A2A2A2A2A2A2A2A2A2A2A2A2A2A2AEC
:100470002A2A2A2A0052582041636B6564202D20C5
:1004800072657665727420737563636573736675E0
:100490006C21002A2A2A2A2A2A2A2A2A2A2A2A2AAD
:1004A0002A2A2A2A2A2A2A2A2A2A2A2A2A2A2A2AAC
:1004B000002A2A2A2A2A2A2A2A2A2A2A2A2A2A2AC6
:1004C0002A2A2A2A2A2A2A2A2A2A2A2A2A2A00528E
:1004D000582041636B6564202D20757064617465DC
:1004E000207375636365737366756C21002A2A2A0D
:1004F0002A2A2A2A2A2A2A2A2A2A2A2A2A2A2A2A5C
:100500002A2A2A2A2A2A2A2A2A2A0056616C696457
:100510002063686F69636573206172653A205B319F
:100520005D2D5B31365D20286368616E6E656C20E1
:10053000312D31362900536574206F7574707574D0
:1005400020666F7220706F727420005B585D2061AE
:10055000626F7274206368616E67657320616E6498
:10056000206578697420525820636F6E6669670051
:100570005B535D20736176652073657474696E6783
:100580007320746F205258005B525D20726576654F
:1005900072742052582073657474696E6773207486
:1005A0006F2064656661756C747300557365206EA9
:1005B000756D62657273205B312D445D20746F2010
:1005C0006564697420706F727473205B452D515D92
:1005D00020666F722073657474696E677300202DD6
:1005E00020726563656976657220636F6E66696700
:1005F000757261746F722C20727820737720000AF4
:100600000A6F70656E4C52536E67200053657420FC
:1006100073657269616C2062617564726174653AB8
:10062000200056616C69642063686F696365733A82
:100630002031202D20342B34202F2032202D203823
:10064000202F2033202D20382B34202F2034202D14
:10065000203132202F2035202D2031322B34202FF5
:100660002036202D20313600536574204368616E9A
:100670006E656C20636F6E6669673A20005365741F
:100680002044617461726174652028302D32293AEA
:10069000200053657420486F70206368616E6E653A
:1006A0006C7320286D61782032342C207365706162
:1006B000726174656420627920636F6D6D61732966
:1006C0002076616C69642076616C75657320312DCC
:1006D0003235353A2000536574206368616E6E656B
:1006E0006C2073706163696E6720287831306B48C5
:1006F0007A293A200053657420524620706F77653E
:10070000722028302D37293A200053657420524634
:10071000206D6167696320286865782920652E67E8
:100720002E20307844454144463030443A2000532E
:1007300065742062617365206672657175656E63AC
:10074000792028696E20487A293A20005B5A5D207A
:10075000656E746572207265636569766572206383
:100760006F6E66696775726174696F6E2075746902
:100770006C79005B465D20646973706C61792061FF
:10078000637475616C206672657175656E63696509
:10079000732075736564005B525D2063616C6375E3
:1007A0006C6174652072616E646F6D206B65792079
:1007B000616E6420686F70206C697374005B495DC2
:1007C000207265696E697469616C697A6520736508
:1007D0007474696E677320746F20736B65746368DB
:1007E0002064656661756C7473005B585D2072658A
:1007F00076657274206368616E67657320616E64EC
:100800002065786974206D656E75005B535D20739B
:100810006176652073657474696E677320746F20E8
:10082000454550524F4D20616E64206578697420B3
:100830006D656E7500557365206E756D62657273BA
:10084000205B302D395D20746F20656469742070E1
:100850006172616D657465727300202D2053797328
:1008600074656D20636F6E66696775726174696F18
:100870006E000A0A6F70656E4C52536E672000510D
:1008800029204F7574707574206265666F726520DB
:100890006C696E6B20283D465329203A2000502970
:1008A00020536C617665206D6F64652028657870D3
:1008B0006572696D656E74616C293A20004F29205C
:1008C00054696D65642042494E44206174207374FC
:1008D000617274757020203A20004E292050504DCE
:1008E000206F7574707574206C696D69746564200F
:1008F000202020203A200044495341424C454400E6
:100900004D292050504D205253534920746F20637D
:1009100068616E6E656C202020203A20004C2920F2
:1009200050504D206D696E696D756D2073796E63E1
:10093000202875732920203A200044495341424C15
:100940004544004B29204661696C736166652062ED
:100950006561636F6E20696E74762E2028312D32AA
:10096000353573293A20004A29204661696C736144
:10097000666520626561636F6E2064656C617920D5
:1009800028302D323535203D3E20313073202D204A
:100990003135306D696E293A200049292046616958
:1009A0006C7361666520626561636F6E206672714B
:1009B0002E203A200048292050574D2073746F7024
:1009C0002064656C6179202020202020203A2000BE
:1009D00047292050504D2073746F702064656C61FE
:1009E00079202020202020203A200046292046611E
:1009F000696C736166652064656C617920202020D4
:100A00002020203A200050574D206368616E6E65AB
:100A10006C200066756E6374696F6E3A2000292041
:100A2000706F72742000506F776572546F776572C3
:100A300000445446205548462033322D62697420C4
:100A400031306368004F70656E4C52536E67525878
:100A5000206D696E6920342F36636800466C7974A6
:100A6000726F6E2F4F72616E6765525820554846FF
:100A70002038636800525820747970653A20004429
:100A8000697361626C656400487A00203D3D200016
:100A900043616C63756C61746564207061636B6540
:100AA0007420696E74657276616C3A200042292068
:100AB0004D6963726F202868616C66292050504D23
:100AC000202020203A00412920496E766572746505
:100AD000642050504D20696E20202020203A0030A4
:100AE00029204D7574652062757A7A657220286DAB
:100AF0006F73746C79293A003929205365726961E2
:100B00006C2062617564726174653A00736D617224
:100B100074506F7274004672536B79005472616E38
:100B200073706172656E740044697361626C6564B0
:100B30000038292054656C656D657472793A2020FF
:100B40002020202020003729204368616E6E656CCC
:100B500020636F6E6669673A202000362920446161
:100B60007461726174652028302D32293A2020206A
:100B700000352920486F70206368616E6E656C7364
:100B80003A2020202020003429204368616E6E65C1
:100B90006C2073706163696E673A202000332920EE
:100BA000524620706F7765722028302D37293A2001
:100BB0002020003229205246206D616769633A2067
:100BC0002020202020202020003129204261736530
:100BD000206672657175656E63793A202020000089
:100BE00000000700020100000304060000000000EE
:100BF00000000001020408102040800102040810D7
:100C00002001020408102004040404040404040263
:100C10000202020202030303030303000000002395
:100C2000002600290000000000250028002B0000FD
:100C3000000000240027002A00002F2E11241FBED0
:100C4000CFEFD8E0DEBFCDBF13E0A0E0B1E0ECE62F
:100C5000F2E602C005900D92A83CB107D9F716E064
:100C6000A8ECB3E001C01D92A239B107E1F71CE086
:100C7000CCE3DCE004C02297FE010E94382FCA3387
:100C8000D107C9F70E946B2E0C9434310C940000EC
:100C900080917705813019F482E080937705809107
:100CA0007705833019F484E0809377050895A8953B
:100CB0000895DC01ED91FC910190F081E02D099502
:100CC00008952091780530917905382748E0C901C9
:100CD000880F991F37FF06C09C0151E2252750E17C
:100CE000352701C09C01415091F73093790520933D
:100CF0007805089588E380937A0580E092ECA1E07E
:100D0000B0E080937B0590937C05A0937D05B09324
:100D10007E0587E08093870580E091EAACEBB3E342
:100D200080937F0590938005A0938105B093820501
:100D300085E0809388058DEE9EEFADEABEED809351
:100D4000830590938405A0938505B0938605E9E813
:100D5000F5E080E090E0863028F4DC01AE54BC4F32
:100D60002C9101C020E0219301968831910599F7DB
:100D700082E08093A1058AE08093A205089580E037
:100D80009EECADEEB4E38093BF059093C005A093B5
:100D9000C105B093C20580E090E0A0E0B0E580938B
:100DA000C3059093C405A093C505B093C605E7ECB1
:100DB000F5E080E081938F5F8031E1F70895A0E056
:100DC000B0E0E5EEF6E00C94012FD82F0E94E02869
:100DD0006115710581059105C9F30E94A42F109238
:100DE0008305109284051092850510928605C4E053
:100DF000812C912C54018A94C0908305D090840555
:100E0000E0908505F0908605FE2CED2CDC2CCC24A2
:100E10000E949F2FA50194010E94E02E6C0D7D1D64
:100E20008E1D9F1D609383057093840580938505B7
:100E300090938605C15001F7DD2309F450C009E8FD
:100E400015E0E801A12CB12C62E3C62ED12CE12CD7
:100E5000F12C8881882309F442C0B39419F40E94CC
:100E60007A063DC00E949F2FA70196010E94E02EA6
:100E7000E1E0E60FA9E8B5E08A2F801B8A1520F48F
:100E80008D918E13F9CFE9CF2091880530E0A0E154
:100E9000B7E20E94782E9B01AC01AE2FB0E00E9419
:100EA000872E40907F05509080056090810570905E
:100EB0008205640D751D861D971D4090BF055090DD
:100EC000C0056090C1057090C205461657066806B9
:100ED000790618F2E993A39488E1A812BACFCDB7A6
:100EE000DEB7E0E10C941D2F8436910520F4BC019F
:100EF00080E090E017C09C018E3B910528F42A55B4
:100F00003109AAE0B0E00CC0823D910528F4245BD1
:100F10003109A4E6B0E004C02D5C3109A8E5B2E0D7
:100F20000E94782EA4E6B0E09B01AC010E94872EBF
:100F3000089590E08C599F4F0E947407089561E0D6
:100F40008AE00E948D2960E08AE00E94C629089507
:100F5000892B11F061E001C060E08AE00E94C6299F
:100F6000089560E08CE00E948D2961E08BE00E9492
:100F70008D2961E08DE00E948D2960E082E00E9471
:100F80008D2961E084E00E948D29089542E050E0BF
:100F900068E476E080E00E9410280895E3E0F0E045
:100FA00089E080935700E491E67081E0E63009F033
:100FB00080E00895CF93DF93C82F0E94CE07882347
:100FC00081F0DFB781E080937605F8940E945706A0
:100FD00088E180936000C0936000C1110E945706B1
:100FE000DFBFDF91CF9108958F929F92AF92BF9212
:100FF000CF92DF92EF92FF92CF93FC01C0A5EC2F2E
:10100000E770F0E0E658FC4FA081B0E0C7FF03C0F6
:1010100024E130E002C02FE030E0FC0197A183E141
:10102000989FF0011124E25CFE4F80809180A280A5
:10103000B380A20FB31F20E43FE14DE750E00E94D0
:10104000922EA50194010E94BE2E8C2F887149F426
:1010500069017A01E0EDCE0EE7E0DE1EE11CF11C35
:101060001BC0C7FF05C060E47AE88CE29EE004C0C4
:1010700060E07EEE8AEB9BE069017A01F8EBCF0E2F
:10108000FBE0DF1EE11CF11CA50194010E94BE2EB5
:10109000C20ED31EE41EF51EC701B60169517C4F76
:1010A0008F4F9F4F28EE33E040E050E00E94BE2E6D
:1010B000A8EEB3E00E94872ECF91FF90EF90DF90D3
:1010C000CF90BF90AF909F908F9008958F3F9105E4
:1010D00051F048F0811522E0920738F081159340D5
:1010E00030F482E0089580E0089581E0089583E07F
:1010F0000895A0E0B0E0EFE7F8E00C940A2FEB01D0
:101100008A01B82FB695A0E028813981F8012083A3
:101110002A813B8121832C813D8122832E813F8145
:101120002383688179814A815B812C813D81EE81B5
:10113000FF819F2F9295990F990F907C272F2370F5
:10114000922B252F2370220F220F922B232F2370F7
:101150002295207F922BF80194830B5F1F4F2896D6
:10116000AF5FBA1788F680FF24C0888199810E94FA
:101170006608D82E8A819B810E946608E82E8C81A1
:101180009D810E946608F82E8E819F810E946608CC
:10119000F0E4DF9EA001112490E1E99E900111246A
:1011A000242B282BE4E0FE9EB0011124262BF8010D
:1011B0002083CDB7DEB7E7E00C94262F803223E002
:1011C000920708F1883E23E0920740F48F51934044
:1011D000E4E096958795EA95E1F70895803D27E04C
:1011E000920718F48C5D93400895883928E092079F
:1011F00068F4885C974074E0969587957A95E1F756
:101200008D509C4F089580E090E008958FEF93E01B
:1012100008958C30910540F4A4E0880F991FAA9599
:10122000E1F7885D9C4F0895843F23E0920718F40E
:1012300084529C4F0895811524E0920740F486570C
:10124000934FF4E0880F991FFA95E1F7089580E92C
:1012500098E008959C013695279525753575821B74
:10126000930B9C0123733373969587959695879579
:1012700083739373820F931F9C0154E036952795D7
:101280005A95E1F7280F391F2F703F7041E051E068
:10129000249FC001259F900D349F900D1124892F0C
:1012A00008952D98882319F000002B9A02C00000A1
:1012B0002B9800002D9A000008952D9A000083B10C
:1012C0002D980000829581700895CF93DF93D82FD9
:1012D0005C9A2D985C98C8E08D2F80780E94510907
:1012E000DD0FC150C9F72D98DF91CF9108958F7709
:1012F0000E9465090895CF93DF93D82FC8E08D2F02
:1013000080780E945109DD0FC150C9F72D98DF91F7
:10131000CF910895CF93DF932D98C8E080E0D82F28
:10132000DD0F0E945D098D0FC150C9F7DF91CF918C
:1013300008950E9477090E948A095C9A0895A1E0A5
:10134000B0E0E5EAF9E00C940F2F806869830E9411
:1013500065096981862F0E947B095C9A2196E2E0EB
:101360000C942B2FCF93C0918305C827E82FF0E072
:10137000E658FA4F678589E70E949F096C2F8DE335
:101380000E949F096C2F82E40E949F09CF910895CB
:1013900086E20E9499090895CF93DF93EC016C8156
:1013A0008CE10E949F096D818DE10E949F096E81F1
:1013B0008EE10E949F096F8180E20E949F096885EB
:1013C00081E20E949F09698582E20E949F096A85E5
:1013D00083E20E949F096B8584E20E949F096C85CD
:1013E00085E20E949F096D858AE20E949F096E85B1
:1013F0008EE60E949F096F858FE60E949F0968898B
:1014000080E70E949F09698981E70E949F096A8994
:1014100082E70E949F09DF91CF910895CF92DF92DA
:10142000EF92FF92CF93DF936B017C01C11488E3AD
:10143000D8068CE9E8068CE1F80628F5C701B60164
:1014400020E836E948E950E00E94BE2EE90168979D
:1014500060E879E687E69FEF0E949A2E6C0D7D1D6D
:101460008E1D9F1DF2E0660F771F881F991FFA954A
:10147000D1F721E732E040E050E00E94BE2EF22E8C
:10148000E32E80E421C0C701B60120E03DE241E344
:1014900051E00E94BE2EE901689760E073ED8EEC8A
:1014A0009EEF0E949A2E6C0D7D1D8E1D9F1D660F56
:1014B000771F881F991F21E732E040E050E00E942B
:1014C000BE2EF22EE32E80E66C2F6F71680F85E73B
:1014D0000E949F096E2D86E70E949F096F2D87E766
:1014E0000E949F09DF91CF91FF90EF90DF90CF9006
:1014F0000895682F8DE60E949F0908958F929F920C
:10150000AF92BF92CF92DF92EF92FF92CF93DF9391
:10151000D82F83E00E9499098093750584E00E948A
:1015200099098093740560E086E00E949F0961E05C
:1015300087E00E949F096FE789E00E949F0965E0AC
:101540008AE00E949F0962E18BE00E949F0965E1A9
:101550008CE00E949F096DEF8DE00E949F0960E082
:101560008EE00E949F09DD2319F08BE291E008C014
:101570002091A10533E1239FC0011124825C9E4F7D
:101580000E94CC096CE880E30E949F096FE082E32F
:101590000E949F0962E483E30E949F098091A20553
:1015A00087FF02C064E101C06AE084E30E949F09F2
:1015B0006AE285E30E949F096DE286E30E949F092B
:1015C00064ED87E30E949F0960E088E30E949F0921
:1015D00060E089E30E949F09D11109C0C090830592
:1015E000D0908405E0908505F090860507C0C5E998
:1015F000CC2EC1ECDC2EED2CCEEDFC2ECAE38F2CD4
:101600009924AA24BB24682D8C2F0E949F09682D41
:1016100085E08C0F0E949F09FE2CED2CDC2CCC2445
:10162000CF5FCE3361F76FEF83E40E949F096FEFC6
:1016300084E40E949F096FEF85E40E949F096FEF89
:1016400086E40E949F09DD2311F066E002C06091EC
:1016500087058DE60E949F0960E089E70E949F0947
:10166000609188058AE70E949F0960E083E70E94F5
:101670009F0960E084E70E949F09D11109C0609131
:101680007F0570918005809181059091820504C04D
:1016900060E071EA8CEB93E30E940E0ADF91CF9138
:1016A000FF90EF90DF90CF90BF90AF909F908F9082
:1016B000089561E087E00E949F0964E28EE70E943E
:1016C0009F0963E088E00E949F0960E088E00E9433
:1016D0009F0965E087E00E949F0962E085E00E9423
:1016E0009F0983E00E9499098093750584E00E9418
:1016F000990980937405089583E00E949909809365
:10170000750584E00E9499098093740561E087E083
:101710000E949F096AE070E080E090E00E94032947
:101720000E94590B00000895CF92DF92FF920F9311
:101730001F93CF93DF931F92CDB7DEB7082F162FDD
:101740008EE399830E949F09F02EC02E9981D92E95
:101750008C2D8F19811738F4F60161916F018FE795
:101760000E949F09F5CF64E085E00E949F0983E015
:101770000E9499098093750584E00E9499098093DD
:1017800074050E94E0286093700570937105809342
:1017900072059093730569E087E00E949F0981E0DC
:1017A000809377050F90DF91CF911F910F91FF905C
:1017B000DF90CF9008950F931F930E94940B809118
:1017C0007705813099F40E94E0280091700510910E
:1017D00071052091720530917305601B710B820BAE
:1017E000930B603A76488140910548F380917705E4
:1017F000813031F46EE971E086EE95E00E94CC2AEA
:101800001F910F9108950F931F9380917705823058
:1018100021F41092770581E020C080917705813016
:10182000D9F40E94E0280091700510917105209173
:10183000720530917305601B710B820B930B613A3B
:1018400076488140910540F061E087E00E949F0961
:101850001092770582E001C080E01F910F910895FA
:10186000CF93DF93EC014AE050E06D2F70E086EEFD
:1018700095E00E949A2B6EE286EE95E00E949E2AE9
:10188000BE0184E0769567958A95E1F76F707727BA
:101890004AE050E086EE95E00E949A2B6EE286EEDA
:1018A00095E00E949E2ABE016F7077274AE050E0C3
:1018B00086EE95E00E949A2BDF91CF910895D82F64
:1018C000C0E0CD1790F45E9A409A64E670E080E044
:1018D00090E00E9403295E98409864E670E080E002
:1018E00090E00E940329CF5FECCF6CE271E080E0D2
:1018F00090E00E940329E4CF0F931F93CF93DF93CF
:10190000EC01062F15E0115051F0CE010E941B3161
:10191000081741F0602FCE010E942331F4CF82E0FE
:101920000E945F0CDF91CF911F910F910895A0E06D
:10193000B0E0EDE9FCE00C94012F482E562EC0E0FB
:10194000D0E0612C712CE12CF12C00E010E0411072
:101950000CC06090D80586E4689E3001112459E1DE
:10196000E52EF12C0EEB15E01EC091E049120FC0E0
:101970006090D805E6E46E9E30011124FBE16F0E05
:10198000711C49E2E42EF12C0AE715E00CC082E05C
:10199000481209C028E1622E77247394EE24E39460
:1019A000F12C07ED15E043018C0E9D1E1092790578
:1019B000109278053401A62CA818B12CC301019609
:1019C0006C01AE14BF04A8F4A00EB11E511006C0E5
:1019D000C3010E941B31F501808305C0F5016081C0
:1019E000C3010E947C0CF50180810E9461063601D2
:1019F000E2CFC301511018C0C3010E941B31B82EA1
:101A0000C6010E941B312B2D30E0322F2227282BBC
:101A100080917805909179058217930779F4C0E059
:101A2000D0E05524539493CF3601609179050E94FC
:101A30007C0C60917805C6010E947C0CC05EDE4F74
:101A4000C13E92E0D90708F482CF852DCDB7DEB72D
:101A5000E0E10C941D2F61E082E00E94970C089554
:101A600060E082E00E94970C8091D705853020F0DD
:101A70001092D7050E942B0D8091D7058093D80531
:101A8000089561E080E00E94970C61E081E00E948F
:101A9000970C089560E080E00E94970C882351F035
:101AA00060E081E00E94970C882321F080917A0504
:101AB000883349F00E94BF060E947A0681E00E94A6
:101AC000DF060E94410D0895882319F06AEA71E04B
:101AD00002C06EEA71E086EE95E00E94CC2A08957D
:101AE000FF920F931F93CF93DF9369EC7BE086EE19
:101AF00095E00E94782A40917F0550918005609181
:101B00008105709182052AE030E086EE95E00E9422
:101B1000A12B63EB7BE086EE95E00E94782A409152
:101B2000830550918405609185057091860520E1BB
:101B300030E086EE95E00E94A12B6DE97BE086EE19
:101B400095E00E94782A4AE050E06091870586EE91
:101B500095E00E94C92B67E87BE086EE95E00E9445
:101B6000782A4AE050E06091880586EE95E00E9470
:101B7000C92B61E77BE086EE95E00E94782AC9E8F0
:101B8000D5E0F12C8E0188818823A9F0FF2031F067
:101B900061EB71E086EE95E00E949B2A21964AE077
:101BA00050E0F801608186EE95E00E94922BF3945C
:101BB000F8E1FF12E7CF86EE95E00E94A62A6BE5DA
:101BC0007BE086EE95E00E94782A4AE050E0609142
:101BD000A10586EE95E00E94C92B66E47BE086EEC7
:101BE00095E00E94782AE091A205E770F0E0EE0F00
:101BF000FF1FEE57FC4F6081718186EE95E00E94D9
:101C0000CC2A61E37BE086EE95E00E94782A809101
:101C1000A2058871883069F028F4811113C068E248
:101C20007BE00CC0803141F0883161F46CE07BE0F6
:101C300005C06CE17BE002C066E17BE086EE95E0EA
:101C40000E94BA2A68EF7AE086EE95E00E94782A30
:101C500040917B0550917C0560917D0570917E05DA
:101C60002AE030E086EE95E00E94A12B6FED7AE04D
:101C700086EE95E00E94782A8091C30580710E94CB
:101C8000640D66EC7AE086EE95E00E94782A8091F9
:101C9000C30580740E94640D6DEA7AE086EE95E0DB
:101CA0000E94782A8091C30580720E94640D60E9C9
:101CB0007AE086EE95E00E94782A8AE795E00E9415
:101CC000F407AB01BC012AE030E086EE95E00E940B
:101CD000832B6BE87AE086EE95E00E94782A8AE70B
:101CE00095E00E94F4079B01AC0160E472E48FE090
:101CF00090E00E94BE2EBA01A9012AE030E086EEF3
:101D000095E00E94832B68E87AE086EE95E00E94D9
:101D1000BA2ACDB7DEB7E5E00C94282F8F929F92B8
:101D2000AF92BF92CF92DF92EF92FF92811107C0E4
:101D30006FE77AE086EE95E00E94BA2A2FC090E025
:101D40000E94740724E630E040E050E00E94BE2E7E
:101D5000CA01B9012AE030E040E050E00E94BE2E06
:101D600049015A016B017C012AE030E0B501A40170
:101D700086EE95E00E94832B6EE286EE95E00E944F
:101D80009E2A2AE030E0B701A60186EE95E00E9487
:101D9000832B63E786EE95E00E94DE2AFF90EF90AA
:101DA000DF90CF90BF90AF909F908F9008951F933A
:101DB000CF93DF9365E77AE086EE95E00E94782A7C
:101DC0008091A305813041F46CE57AE086EE95E0E0
:101DD0000E94BA2A10E050C0823019F465E47AE01B
:101DE000F5CF843019F461E37AE0F0CF853091F7D4
:101DF00066E27AE0EBCFC12FD0E0C930D1050CF418
:101E000041C068E3610F86EE95E00E949E2A6EE174
:101E10007AE086EE95E00E94782ABE016F5F7F4FE0
:101E20004AE050E086EE95E00E94622B63E17AE0A2
:101E300086EE95E00E94782ACD55DA4FE981E032AE
:101E400018F566E07AE086EE95E00E94782A8981AE
:101E5000803130F06DE673E086EE95E00E949B2ABB
:101E600069816F7070E06F5F7F4F4AE050E086EEEF
:101E700095E00E946B2B1F5F80914C05181708F4AA
:101E8000BACF0FC061E3BECFEF70F0E0EE0FFF1FDF
:101E9000EE56FC4F6081718186EE95E00E94CC2A5F
:101EA000EACF6BEE79E086EE95E00E94782A809189
:101EB000BB050E948E0E60ED79E086EE95E00E94F3
:101EC000782A8091BC050E948E0E65EB79E086EE43
:101ED00095E00E94782A8091BD050E948E0E6AE9E5
:101EE00079E086EE95E00E94782A4091B305509102
:101EF000B4056091B5057091B605411551056105B0
:101F0000710539F12AE030E086EE95E00E94A12BC0
:101F100067E679E086EE95E00E94782A8091B70521
:101F20000E949907AB01BC012AE030E086EE95E003
:101F30000E94A12B63E479E086EE95E00E94782A66
:101F40004AE050E06091B80586EE95E00E94C92B0A
:101F500006C06AE379E086EE95E00E94BA2A6DE158
:101F600079E086EE95E00E94782A6091B90570913B
:101F7000BA054AE050E086EE95E00E94B32B60E09F
:101F800079E086EE95E00E94782A6091B20560348F
:101F900050F470E06F5F7F4F4AE050E086EE95E0CE
:101FA0000E946B2B06C067EF78E086EE95E00E94FA
:101FB000BA2A6AED78E086EE95E00E94782A809150
:101FC000B10580FF03C063EB71E002C067EB71E015
:101FD00086EE95E00E94CC2A6DEB78E086EE95E0E7
:101FE0000E94782A8091B10582700E94640D6EE98A
:101FF00078E086EE95E00E94782A8091B1058470A1
:102000000E94640D6FE778E086EE95E00E94782AE2
:102010008091B10588700E94640DDF91CF911F916E
:1020200008950F931F93CF93DF93209149052F3F7E
:10203000A9F56FEF75E086EE95E00E94782A88E8B2
:1020400093E00E94300C6EED75E086EE95E00E9404
:10205000782A80914A0590914B050E94300C6BEADA
:1020600075E086EE95E00E94BA2A68E875E086EE93
:1020700095E00E94BA2A60E775E086EE95E00E943E
:10208000BA2A6BE475E086EE95E00E94BA2A86EEE5
:1020900095E00E94A62A0E94D70E68C012160CF086
:1020A00065C0332727FD309580914C0590E082175D
:1020B00093070CF45BC066E375E086EE95E00E9442
:1020C000782A60914905772767FD70954AE050E0CE
:1020D00086EE95E00E946B2B6BE075E086EE95E056
:1020E0000E94782A10E008E280914D051817D0F57B
:1020F000C12FD0E0CC0FDD1FC25BDA4F288130E06A
:1021000080914905992787FD9095019728173907F0
:1021100039F56BEB71E086EE95E00E949B2A4AE070
:1021200050E0602F86EE95E00E94922B6FEB71E0FD
:1021300086EE95E00E949B2AE981EF70F0E0EE0FB9
:10214000FF1FEE56FC4F6081718186EE95E00E9484
:102150009B2A63EC71E086EE95E00E949B2A0F5F5C
:102160001F5FC2CF86EE95E00E94A62ADF91CF9135
:102170001F910F910895FF920F931F93CF93DF93B9
:10218000C9E8D5E0F12C8E0188818823D1F165EC76
:1021900071E086EE95E00E949B2A4AE050E06F2DA8
:1021A00086EE95E00E94922B62ED71E086EE95E05E
:1021B0000E949B2A2196F801208130E0A0E1B7E23D
:1021C0000E94782E9B01AC01A0918805B0E00E948E
:1021D000872EAB01BC0180917F0590918005A09175
:1021E0008105B0918205480F591F6A1F7B1F2AE0A5
:1021F00030E086EE95E00E94A12BF394F8E1FF1207
:10220000C2CFCDB7DEB7E5E00C94282F1092E304DF
:1022100085E6E4EEF4E0DF011D928A95E9F7089582
:10222000CF93C82F8F3719F0883009F045C0E0915F
:10223000E304EE23D9F1E150E093E304F0E0EC5144
:10224000FB4F10826DE070E086EE95E00E9459062B
:10225000C0E08091E304C81760F4EC2FF0E0EC518B
:10226000FB4F608170E086EE95E00E945906CF5FDB
:10227000F0CF60E270E086EE95E00E9459066DE0D6
:1022800070E086EE95E00E945906C0E08091E3047C
:10229000C81778F5EC2FF0E0EC51FB4F608170E04F
:1022A00086EE95E00E945906CF5FF0CF67E086EE9C
:1022B00095E00E949E2A1DC08B3119F40E940611E0
:1022C0001AC08D30C1F08A30B1F08091E3048436B9
:1022D00068F76C2F70E086EE95E00E945906E09159
:1022E000E30481E08E0F8093E304F0E0EC51FB4FB8
:1022F000C08380E001C081E0CF910895CF93C82FC3
:102300000E94E0286093CC047093CD048093CE04A7
:102310009093CF04C093E104CC2329F040E051EE28
:1023200060E070E004C040E855E260E070E086EEF6
:1023300095E00E94282DCF9108959091D004492FC7
:102340004F7050E0BA016F5F7F4F292F30E0E4E01B
:1023500035952795EA95E1F76217730759F0FA0169
:10236000EF52FB4F808381E0890F8F70907F892B24
:102370008093D00408956EE770E086EE95E00E94A9
:1023800059060895A3E1B1E0E8ECF1E10C94022FC5
:10239000E9E8F5E0712C8191882321F0739428E11C
:1023A0007212F9CF66ED71E086EE95E00E94CC2ABC
:1023B0004AE050E0672D86EE95E00E94C92B80E050
:1023C0000E947E0A0E94590B8E010E5F1F4FC12C86
:1023D000D12C7601C39466246A945C2C0E94D42884
:1023E0004B015C012091880530E0A0E1B7E20E943A
:1023F000782E9B01AC01C701B6010E949A2E209154
:102400007F05309180054091810550918205620FD2
:10241000731F841F951F2091BF053091C005409107
:10242000C1055091C205261737074807590718F408
:10243000F801608229C08C2D0E94B20961E070E031
:1024400080E090E00E940329F80110820E94D428C5
:10245000681979098A099B09643F714081059105D2
:1024600040F40E94C809F8019081981778F780839A
:10247000EDCF50FE05C05D9841985E9A409A04C029
:102480005D9A419A5E9840982FEFC21AD20AE20AEA
:10249000F20A0F5F1F4F8FEFC816D104E104F10459
:1024A00009F09BCFCE019395FC01D82E7FEF68EC0D
:1024B0002E2F281B271510F051E056C0DE01129672
:1024C00051E02FEF41E03D91321710F0322F01C063
:1024D000452F5F5F5F3F11F0232FF5CF4193242FEE
:1024E00030E0A1E0B0E0AC0FBD1FA20FB31F5C93C2
:1024F000413079F0DE01A20FB31F5C93423049F006
:10250000AFEFBFEFAC0FBD1FA20FB31F6C934E3FD9
:1025100078F6A2E0B0E0AC0FBD1FA20FB31F7C9312
:102520004D3F30F6A3E0B0E0AC0FBD1FA20FB31FCC
:102530006C93BECF452F242F30E0FC01E20FF31F38
:102540006081AFEFB0E0AC0FBD1FA20FB31F2C91A5
:10255000621748F44150DC01A40FB11D2C91208377
:102560006C934111E8CF5F5F571520F3372D3695F7
:1025700020E0231770F4DC01A20FB11D4C91522F03
:10258000530FFC01E50FF11D50815C9340832E5FDA
:10259000F0CFF9E8EF2EF5E0FF2E8C01802F8D199A
:1025A000871598F4F801C1908F014AE050E06C2D36
:1025B00086EE95E00E94922B6CE286EE95E00E94FA
:1025C0009E2AF701C1927F01E9CF86EE95E00E9435
:1025D000A62A81E0CD5EDE4FEFE00C941E2F1F9205
:1025E0000F920FB60F9211241F932F933F934F9387
:1025F0005F936F937F938F939F93AF93BF93CF938B
:10260000DF93EF93FF93C0918600D0918700809174
:102610008704909188042091A904211155C09E013E
:10262000281B390B8091C3059091C405A091C50565
:10263000B091C60585FD02C036952795253C49E039
:102640003407B8F140910A0150E060E070E02CE1FD
:10265000B695A795979587952A95D1F70097A105E7
:10266000B10521F481E090E0A0E0B0E08417950787
:10267000A607B707D8F480910A018F3FB9F040E070
:1026800080910A01481780F4842F90E0880F991FE9
:10269000FC01E757FB4F20813181FC01E55FFE4FD4
:1026A000318320834F5FECCF1092AA0410920A016D
:1026B0000BC02D3B82E0380720F080910A01803169
:1026C000D8F08FEF80930A01D0938804C0938704D9
:1026D000FF91EF91DF91CF91BF91AF919F918F913A
:1026E0007F916F915F914F913F912F911F910F902B
:1026F0000FBE0F901F90189510910A0181E0810F75
:1027000080930A01C9010E94DE08E12FF0E0EE0F7C
:10271000FF1FE757FB4F91838083D6CF83E08093E1
:1027200080008AE9809381008091C30586FD05C001
:10273000809181008064809381008FEF9FEF909360
:1027400089008093880080916F00806280936F0081
:1027500008950E94300D8091D805843011F41092B4
:10276000D80508956F3018F086958058089589E04F
:10277000689F802D11240895A0E0B0E0E2ECF3E121
:102780000C94092FC82F0E94E02800913804109162
:10279000390420913A0430913B046B017C01C01A4A
:1027A000D10AE20AF30A9701860149E8C41643E117
:1027B000D406E104F10410F010923C046093380454
:1027C0007093390480933A0490933B042091A904B8
:1027D0008FEF820F8230E8F5E0913C04EE2309F49C
:1027E0006EC1E13011F482E0D8C1E03178F581E0CA
:1027F0008E0F80933C04F0E0E757FB4FC08380319D
:1028000009F0D4C1EBE8F4E0213029F4A181A695C8
:10281000A695808108C080819181A92FA695A69553
:10282000A69596958795A03148F4B0E090E0AA0F60
:10283000BB1FA55FBE4F11969C938E931092AA0466
:10284000329684E0E939F807F9F6B0C110923C04F9
:10285000ADC1233009F023C1E0913C04E11118C05F
:10286000CF3009F011C10E94D4280091B704109113
:10287000B8042091B9043091BA04601B710B820B2B
:10288000930B623071058105910508F089C1FCC088
:10289000E83148F481E08E0F80933C04F0E0E85783
:1028A000FB4FC083F1C0E83109F0ECC0C111EAC0B0
:1028B00040E050E0ABE0CA01B3E0880F991FBA9541
:1028C000E1F7A49F9001A59F300D1124F901E7576E
:1028D000FB4F6081E1817E2F777075956795FC01D4
:1028E000EE0FFF1FE55FFE4F71836083F901E6572E
:1028F000FB4FB081B695B695B695E181FE2FF29566
:10290000FF0FF07E6F2F6B2BE695E695E6957E2FF9
:10291000777075956795FC01EE0FFF1FE35FFE4F23
:1029200071836083F901E557FB4FB081B295B6958D
:10293000B695B370C181DC2FDD0FDD0F6D2F6B2BD2
:10294000C295C695C695C370E281E170EE0FEE0F99
:102950007E2F7C2B75956795FC01EE0FFF1FE15FC5
:10296000FE4F71836083F901E357FB4FB081B69549
:10297000E181FE2FF795FF27F7956F2F6B2BE695DB
:102980007E2F777075956795FC01EE0FFF1FEF5E48
:10299000FE4F71836083F901E257FB4FB081B2951E
:1029A000BF70E181FE2FF295F07F6F2F6B2BE295C8
:1029B000EF707E2F777075956795FC01EE0FFF1F06
:1029C000ED5EFE4F71836083F901E157FB4FB081EB
:1029D000BB1FBB27BB1FC181DC2FDD0F6D2F6B2BF6
:1029E000CC1FCC27CC1FE281E370EE0F7E2F7C2B17
:1029F00075956795FC01EE0FFF1FEB5EFE4F71832F
:102A00006083F901EF56FB4FB081B695B695E18131
:102A1000FE2FF295FF0FFF0FF07C6F2F6B2BE695CB
:102A2000E6957E2F777075956795FC01EE0FFF1F79
:102A3000E95EFE4F71836083F901EE56FB4F208102
:102A40002295269527703181E32FEE0FEE0FEE0FC2
:102A50006E2F622B732F72957695777075956795AB
:102A6000FC01EE0FFF1FE75EFE4F718360834F5F37
:102A70005F4F4230510509F01ECF80919F0483FFC4
:102A80001092AA0410923C040E94D4286093B704C8
:102A90007093B8048093B9049093BA0487C024302B
:102AA00009F084C060913C0461110BC0C83AB1F4D4
:102AB000109279051092780588EA0E94610681E0FB
:102AC0006CC0613019F4C093370404C0623031F433
:102AD000C09336048C2F0E9461065AC0E0913604E0
:102AE0002E2F30E0220F331F462F50E0C9010296EF
:102AF000841795073CF0633268F7FA01EA57FB4FF9
:102B0000C083E8CF2D5F3F4F8C2F90E06091780518
:102B1000709179054217530749F4982F8827862723
:102B20009727909379058093780532C068177907C5
:102B300069F580913704813049F5E13118F080E181
:102B400080933604F0903604CAE8D4E000E010E048
:102B50000F15D0F4FE013197808190E0982F8827DF
:102B60002881822B63E0969587956A95E1F70E940C
:102B7000DE08F801EE0FFF1FE55FFE4F91838083B3
:102B80000F5F1F4F2296E4CF1092AA0410923C04CC
:102B900080913C04882351F08F5F80933C0406C0F1
:102BA00080913C048F5F80933C046ECFCDB7DEB73D
:102BB000E8E00C94252FE82FF0E0E254FA4FE1858D
:102BC000E03150F4F894F0E0EE0FFF1FE55FFE4FA8
:102BD00080819181789408958EE08E0F8B3058F427
:102BE000F0E0E25FF10924E62E9FC0012F9F900DD7
:102BF00011240C960895E03FF1F028F4E03161F0E3
:102C0000E13161F006C0ED3F81F0EE3F89F0E13F38
:102C100049F080E092E0089582E101C083E10E94E2
:102C2000222A089586E090E008958AEF93E00895BF
:102C30008FEF93E0089580E090E00895A2E2B0E085
:102C4000E4E2F6E10C94FF2E9E012F5F3F4F80E1FE
:102C5000D9011D928A95E9F764E072E086EE95E06D
:102C600029A33AA30E94CC2A0E947C0B1D8A1E8AAB
:102C70001F8A188E312C212C00E0812C912C5401BC
:102C8000412C74E7572E7BE8672E72E3772EE0E540
:102C9000CE2EE3ECDE2EE12CF12C84EF91E0A0E0CF
:102CA000B0E08D8F9E8FAF8FB8A380E09EECADEE2D
:102CB000B4E3898F9A8FAB8FBC8F80E094E7ABE849
:102CC000B2E3898B9A8BAB8BBC8B86EE95E00E942E
:102CD000E02B892B09F4E1C086EE95E00E940D2CD3
:102CE0009C0133272C32310509F442C0ACF4233265
:102CF000310509F0ABC019821A821B821C821D8229
:102D00001E821F82188619861A861B861C861D86BF
:102D10001E861F86188A60C02434310529F02335A9
:102D2000310509F4B2C092C064E486EE95E00E94D9
:102D30009E2A2AE030E040E054E76BE872E386EE3A
:102D400095E00E942C2B6CE286EE95E00E949E2A74
:102D50002AE030E040E05EEC6DEE74E386EE95E054
:102D60000E942C2B6CE286EE95E00E94DE2AADCF0D
:102D70000F5F043009F0A9CF29813A814B815C8132
:102D8000A8EEB3E00E94872E698B7A8B8B8B9C8B8D
:102D90002D813E814F8158850E94872E698F7A8FC1
:102DA0008B8F9C8F29853A854B855C852D8F3E8F37
:102DB0004F8F58A32D853E854F8558890E94872EB9
:102DC0006B017C0160323EE473078105910530F4AC
:102DD00062E38CE10E949F0900E077CF603345E712
:102DE00074078105910510F462E2F3CF60345CE969
:102DF00075078105910510F466E2EBCF80E5C816F2
:102E000083ECD806E104F10410F462E1E2CF90E62D
:102E1000C9169AEED906E104F10410F465E1D9CFA0
:102E2000A0E7CA16A1E1DA06A1E0EA06F10410F46F
:102E300061E0CFCFB0EACB16B6E8DB06B1E0EB0637
:102E4000F10410F463E0C5CF65E0C3CF10ED180FB7
:102E50001A3008F03ACFE1E0F0E0EC0FFD1F24E07B
:102E6000029FE00DF11D11242081318142815381A7
:102E7000AAE0B0E00E94872E610F711D811D911D97
:102E8000608371838283938320CF49885A886B88BB
:102E90007C88812C912C540118CF81149104A104B9
:102EA000B10489F4C301B2010E940E0A61E070E02E
:102EB00080E090E00E9403291D8A1E8A1F8A188ED6
:102EC000312C22242A948D8D9E8DAF8DB8A1881629
:102ED0009906AA06BB06D0F40E94C8092D893E892E
:102EE0004F89588D280F311D411D511D2D8B3E8B53
:102EF0004F8B588F381608F4382E821508F4282E78
:102F00003FEF831A930AA30AB30A56C0C301B20162
:102F100028EE33E040E050E00E94BE2EBA01A90145
:102F20002AE030E086EE95E00E94832B6CE286EE8C
:102F300095E00E949E2A4AE050E0632D86EE95E0DF
:102F40000E94922B6CE286EE95E00E949E2A6D898B
:102F50007E898F89988DA50194010E94BE2EBA01A9
:102F6000A9012AE030E086EE95E00E94832B6CE216
:102F700086EE95E00E949E2A4AE050E0622D86EEA1
:102F800095E00E94922B6CE286EE95E00E94DE2A8C
:102F90004C0C5D1C6E1C7F1C898D9A8DAB8DBC8D7D
:102FA00084159505A605B70520F449885A886B88CD
:102FB0007C88812C912C540129893A894B895C8920
:102FC000283E33404105510509F07FCEA296E2E14B
:102FD0000C941B2FACE1B0E0E0EFF7E10C94092F6B
:102FE0000E94E0286B017C0181E00E947E0A14E7C8
:102FF00003E0198361E0CE0101960E94DB0B009390
:1030000077050E94590B6AEF70E080E090E00E9423
:10301000032980917705833089F486EE95E00E943C
:10302000E02B892B59F40E94E0286C197D098E0948
:103030009F096038734C894C9140D8F28091770594
:10304000833009F44FC08FE70E9477090E948A09F4
:103050008983843511F083E05CC00E948A09109254
:103060004A0580934B050E948A0920914A053091B8
:103070004B05280F311D30934B0520934A050E94C4
:103080008A0980934C050E948A0980934D058131FD
:1030900010F7F12C0F2D10E080914D0590E0880F76
:1030A000991F0817190740F40E948A09F801E25B8A
:1030B000FA4F8083F394EECF80E7898361E0CE01FD
:1030C00001960E94DB0B83E0809377050E94590BE9
:1030D00062E370E080E090E00E9403298091770530
:1030E000833011F482E015C08FE70E9477090E94B7
:1030F0008A098983803509F0AECF03EA15E00E9482
:103100008A09F80181938F01F5E00E3B1F07B9F79B
:1031100081E06C96E8E00C94252F80914905992771
:1031200087FD9095A92FB92FFC013196EB30F10561
:1031300008F066C0EC5CFF4F0C94362F62E778E035
:1031400086EE95E00E94BA2A88E893E00E94300C4F
:103150006AE578E086EE95E00E94BA2A65E378E0B9
:1031600086EE95E00E94BA2A6BE078E086EE95E064
:103170000E94BA2A6AEE77E086EE95E00E94BA2AAB
:103180006DEB77E086EE95E00E94BA2A67E977E07A
:1031900086EE95E00E94BA2A63E777E086EE95E036
:1031A0000E94BA2A6CE477E086EE95E00E94BA2A83
:1031B00086EE95E00E94A62A0E94700D21C06FE263
:1031C00077E01AC06AE077E017C065EF76E014C0D8
:1031D00066ED76E011C062E976E00EC06DE776E05C
:1031E0000BC068E676E086EE95E00E94BA2A62E2BD
:1031F00076E002C06CE076E086EE95E00E94BA2AA6
:103200006AE070E080E090E00E94032986EE95E09D
:103210000E94E02B892B29F086EE95E00E940D2C70
:10322000F5CF0895ACE1B0E0E8E1F9E10C94092FA5
:10323000909149059F3F09F023C1482F50E0FA01C2
:103240003A97EF36F10508F00FC1E15CFF4F0C949F
:10325000362F61E172E0A0C06DE172E086EE95E08C
:103260000E94CC2A85E789838BE1E3EAF5E0DE0161
:10327000129601900D928A95E1F76CE1CE010196CC
:103280000E94DB0B0E94590B83E08093770568EC6A
:1032900070E080E090E00E940329809177058430FF
:1032A00009F0E2C08FE70E9477090E948A098983AA
:1032B000853509F0D9C06DEE74E086EE95E00E9488
:1032C000BA2A6FEC74E086EE95E00E94BA2A61EBB0
:1032D00074E096C065E372E086EE95E00E94CC2A29
:1032E00089E6898361E0CE0101960E94DB0B0E9492
:1032F000590B83E08093770568EC70E080E090E004
:103300000E94032980917705843009F0ADC08FE7D2
:103310000E9477090E948A0989838E010E5F1F4FE0
:103320007E014DE1E40EF11C0E948A09F8018193AF
:103330008F01EE15FF05C1F78BE1FE013296A3EA7E
:10334000B5E001900D928A95E1F78981893409F001
:103350008BC063E974E086EE95E00E94BA2A65E7C7
:1033600074E086EE95E00E94BA2A67E574E048C0F2
:103370006FE472E086EE95E00E94CC2A8EEF809397
:10338000490572C080528750805390914C05981720
:1033900008F066C06EE572E086EE95E00E94CC2AE9
:1033A00063C084E18093490560E274E029C085E14F
:1033B0008093490569EE73E023C086E18093490557
:1033C00062EB73E01DC087E18093490568E673E016
:1033D00017C088E18093490567E573E011C089E172
:1033E0008093490563E473E00BC08AE1809349054B
:1033F0006EE273E005C08BE18093490566E073E0FF
:1034000086EE95E00E94BA2A2FC06CEE72E086EE3E
:1034100095E00E94BA2A8091B10591E01DC066ED49
:1034200072E086EE95E00E94BA2A8091B10592E0A2
:1034300013C061EC72E086EE95E00E94BA2A80919A
:10344000B10594E009C066EA72E086EE95E00E945C
:10345000BA2A8091B10598E089278093B1058FEF52
:10346000809349050E94111086EE95E00E94E02BA2
:10347000892B09F45AC186EE95E00E940D2CF4CFF9
:103480000E941011882309F450C18091E304811136
:1034900004C08FEF8093490540C140E050E060E0F8
:1034A00070E084EE94E00E94AD2F40914905042F16
:1034B000112707FD1095212F312FF8013197EB319E
:1034C000F10508F01AC1E255FF4F0C94362F55272D
:1034D00047FD509520914C0530E0241735070CF43A
:1034E0000CC18B019C0101501109210931090032E5
:1034F00011052105310558F0C0904D05EFE4F5E0C8
:10350000F12CD12CA8E2EA2E415051090FC0FA014A
:10351000ED55FA4F61506083D8C0DF0111972C91AF
:1035200030E02417350729F0F3943296FC10F5CFDC
:10353000CAC00E2D10E020E030E00617170728075C
:10354000390741F42081DA01AD55BA4F11962C9319
:10355000DD24D394E394E8CF6F3F71058105910595
:1035600011F008F0CAC06093BB05AFC06F3F710592
:103570008105910511F008F0C0C06093BC05A5C09D
:103580006F3F71058105910511F008F0B6C0609399
:10359000BD059BC02091E40420622037E9F440E09F
:1035A00050E060E070E085EE94E00E94AD2F9B015A
:1035B000AC01DC01CB010197A109B1090897A10574
:1035C000B10508F0ADC0A4EDB0E30E94872E6A5E9D
:1035D0007C4A8A46954E24C02636E9F440E050E005
:1035E00060E070E085EE94E00E94AD2F9B01AC019D
:1035F000DC01CB010197A109B1090797A105B1052C
:1036000008F08EC0A8EAB1E60E94872E645E7C4373
:103610008E46944E05C0611571058105910571F0C6
:103620008B019C0114572B4832430130FAE51F07E8
:10363000F2E62F07F2E03F0708F05FC06093B305A2
:103640007093B4058093B5059093B6053EC06F3F67
:1036500071058105910511F008F04FC06093B70521
:1036600034C08B019C0101501109210931090F3F20
:1036700011052105310508F040C06093B80525C04B
:103680008B019C01045C1940210931090D344DE185
:1036900014072105310528F47093BA056093B90524
:1036A00014C0611571058105910521F48FEF809398
:1036B000B2050BC06134710581059105F0F46150CC
:1036C0006093B20502C0DD20C1F08091E204811157
:1036D0001AC08091830590918405A0918505B091D1
:1036E00086050196A11DB11D8093830590938405E5
:1036F000A0938505B093860506C060E772E086EE6C
:1037000095E00E94CC2A0E9406118FEF8093490514
:103710006AE086EE95E00E94DE2A0E94111005C044
:1037200061E070E080E090E07BCF6C96E8E00C9484
:10373000252F6AE572E086EE95E00E94BA2A62E4DF
:1037400072E086EE95E00E94BA2A86EE95E00E942D
:10375000E02B892B31F086EE95E00E940D2C0E9423
:1037600012190E94EA17823029F0833051F46DE07B
:1037700072E002C064E272E086EE95E00E94BA2A2E
:1037800008958FEF809349051092E2040E94111072
:10379000809149058E3F69F086EE95E00E94E02B0E
:1037A000892BB1F386EE95E00E940D2C0E94121930
:1037B000EFCF08950F931F93109149051F3F09F014
:1037C000D2C0893409F457C000F5883309F469C0C0
:1037D00058F4803309F477C008F061C08B3109F4E4
:1037E00040C08132B1F1B9C0813409F487C030F4EE
:1037F000893309F466C0803461F1AFC0823409F4C2
:103800008EC0863409F448C0A8C0823609F487C047
:1038100078F4883531F128F48235C1F18335E1F04F
:103820009CC08A3509F494C0813609F467C095C0FC
:10383000823761F128F4863679F18936E1F08DC05E
:10384000883779F08A3709F483C0833709F085C057
:1038500003C061E172E015C00E94410D6EE872E0A4
:1038600004C00E944A0D68EA72E086EE95E00E946C
:10387000CC2A8EEF70C00E947A060E94BF0667ECC9
:1038800072E086EE95E00E94CC2A67C081E00E943B
:10389000DF0660EE72E0F5CF0E94BB105EC0805381
:1038A0005AC06AEF71E086EE95E00E94BA2A9091C4
:1038B000A20588E0890F8871977E892B8093A205E5
:1038C0001AC089E048C067EE71E086EE95E00E947C
:1038D000BA2A8091C3059091C405A091C505B09105
:1038E000C60520E182278093C3059093C405A09369
:1038F000C505B093C605109349052FC061ED71E071
:1039000086EE95E00E94BA2A8091C3059091C40585
:10391000A091C505B091C60540E4842710C060ECB5
:1039200071E086EE95E00E94BA2A8091C3059091DD
:10393000C405A091C505B091C60520E282278093F9
:10394000C3059093C405A093C505B093C60502C0F6
:103950000E94991B8FEF80934905809149058E3F06
:1039600009F0D4C0DDC00E941011882309F4D8C02A
:103970008091E304811104C08FEF80934905C6C094
:1039800040E050E060E070E084EE94E00E94AD2FF3
:1039900000914905112707FD1095212F312FF801BE
:1039A0003197E930F10508F0B4C0E753FF4F0C94AC
:1039B000362F8B019C01015014472B4832430F3F97
:1039C00019452246324008F0A4C060937F057093E9
:1039D0008005809381059093820577C0609383056D
:1039E00070938405809385059093860581E080938C
:1039F000E2046BC0683071058105910508F089C04B
:103A00006093870562C08B019C0101501109210957
:103A100031090A3011052105310508F07AC060939B
:103A2000880553C061EB71E084EE94E00E94E730BA
:103A300010E0009799F00E94C130009779F018319A
:103A400030F4E12FF0E0E658FA4F87871F5F61EB13
:103A500071E080E090E00E94E730EBCF1831A8F5EC
:103A6000E12FF0E0E658FA4F17861F5FF7CF653079
:103A700071058105910508F04CC06093A10525C032
:103A80008B019C01015011092109310906301105F2
:103A900021053105F0F52091A205287F262B2093E2
:103AA000A20513C08B019C010150110921093109A4
:103AB0000115124C2140310560F560937B05709330
:103AC0007C0580937D0590937E058091E2048111B1
:103AD00013C08091830590918405A0918505B091D4
:103AE00086050196A11DB11D8093830590938405E1
:103AF000A0938505B09386050E9406118FEF8093F1
:103B000049056AE086EE95E00E94DE2A0E948D1843
:103B100007C060E772E086EE95E00E94CC2AECCF09
:103B20001F910F9108958FEF809349051092E20441
:103B30000E948D18809149058E3F69F086EE95E0D0
:103B40000E94E02B892BB1F386EE95E00E940D2CAC
:103B50000E94DA1BEFCF6AE070E080E090E00E9404
:103B6000032986EE95E00E94E02B892B29F086EE52
:103B700095E00E940D2CF5CF0895CF93C82F682FA4
:103B800086EE95E00E943A2C90916E059C279093CA
:103B90006E05CF910895A1E0B0E0E1EDFDE10C9458
:103BA0000F2F99830E94BD1D9981892F0E94BD1DF1
:103BB0002196E2E00C942B2F1F93CF93DF93182FC5
:103BC000EB0110926E0565EB70E086EE95E00E94C9
:103BD000590662E670E086EE95E00E945906812F54
:103BE0000E94BD1DCE010E94CB1DDF91CF911F9180
:103BF000089560916E0586EE95E00E943A2C089536
:103C0000A1E2B0E0E6E0FEE10C940B2F7B018A011B
:103C10008C3009F453C108F040C0863009F4BCC0B0
:103C200018F5833009F491C070F4813009F472C042
:103C3000823009F04AC26BE170E082E00E94DC1D34
:103C400003EA15E078C0843009F487C0853009F0B4
:103C50003CC260914D0570E0660F771F85E00E94C1
:103C6000DC1D0EE415E086C0893009F4A7C070F4AD
:103C7000873009F49BC0883009F027C261E070E00A
:103C800088E00E94DC1D8091D80525C28A3009F4A5
:103C9000CAC08B3009F4F2C018C28A3609F475C163
:103CA000D8F4873609F43AC138F4853609F40EC1E0
:103CB000863609F41FC109C2883609F437C189362E
:103CC00009F003C261E070E089E60E94DC1D0E94F9
:103CD0007A060E94BF06F7C18D3609F4D4C138F4C4
:103CE0008B3609F491C18C3609F49AC1EEC18E3637
:103CF00009F4DEC1873C09F0E8C161E070E087ECBF
:103D00000E94DC1D81E00E94BD1D0E94F91D1092E1
:103D10006F05E5C169E270E081E00E94DC1D0AE701
:103D200015E0F80181918F010E94BD1DF5E0033A75
:103D30001F07B9F7D2C1F80181918F010E94BD1D03
:103D4000F5E00E3B1F07B9F7C8C161E070E083E002
:103D50000E94DC1D0E94EA17BEC161E070E084E0B1
:103D60000E94DC1D81E00E94BD1D0E94F91D0E9481
:103D70001E16B5C180914D0590E0880F991F9801DE
:103D80002E5435402817390708F0A7C1F801819152
:103D90008F010E94BD1DEECF62E070E086E00E94C0
:103DA000DC1D88E893E00E94CB1D97C161E070E0C4
:103DB00087E00E94DC1D80914C058DC186E68983D9
:103DC00061E0CE0101960E94DB0B0E94590B83E05B
:103DD0008093770568EC70E080E090E00E94032912
:103DE000809177058430D9F48FE70E9477090E948B
:103DF0008A098983863469F460E270E089E00E9470
:103E0000DC1D10E20E948A090E94BD1D1150D1F7ED
:103E100064C161E070E089E00E94DC1D54C161E092
:103E200070E089E055C169E170E08AE00E94DC1D24
:103E300081E08093BE05209176058091C305909125
:103E4000C405A091C505B091C605222311F0806874
:103E500001C08F778093C3059093C405A093C505D7
:103E6000B093C6050EEB15E0F80181918F010E9419
:103E7000BD1DF5E0073D1F07B9F72FC161E270E0F6
:103E80008BE00E94DC1D8091AA048F3F39F0809165
:103E9000AA0491E0980F9093AA0402C08091AA040A
:103EA0000E94BD1D10E0812F0E94DB150E940909B0
:103EB0000E94CB1D1F5F1031B1F70FC161E070E0B0
:103EC0008CE00E94DC1D8091D70505C161E070E0A7
:103ED00085E60E94DC1D89E2E816F10409F0FAC0CB
:103EE000D801EAE7F5E08D91819385E0E33AF807A0
:103EF000D1F7E9C061E070E086E60E94DC1DEBE1ED
:103F0000EE16F10409F0E6C0D801E3EAF5E08D9180
:103F1000819385E0EE3BF807D1F7D5C061E070E012
:103F200087E60E94DC1D0E94410DCDC061E070E07B
:103F300088E60E94DC1D85E789838BE1E3EAF5E0F2
:103F4000DE01129601900D928A95E1F76CE1CE01A7
:103F500001960E94DB0B0E94590B83E0809377054A
:103F600060E273E080E090E00E9403298091770591
:103F7000843009F0AFC08FE70E9477090E948A0958
:103F80008983853509F0A6C09EC061E070E08AE6AD
:103F90000E94DC1D89E6898361E0CE0101960E94C2
:103FA000DB0B0E94590B83E08093770560E273E09E
:103FB00080E090E00E94032980917705843009F029
:103FC00089C08FE70E9477090E948A0989838E0140
:103FD0000E5F1F4F7E01EDE1EE0EF11C0E948A097B
:103FE000F80181938F01EE15FF05C1F78BE1FE010A
:103FF0003296A3EAB5E001900D928A95E1F78981A6
:10400000893409F067C05FC061E070E08BE60E9410
:10401000DC1DF80180818093D8050E944A0D53C0B1
:1040200061E070E08CE60E94DC1DF0E2EF16F10426
:1040300061F487E6898380E2F801DE01129601903F
:104040000D928A95E1F761E203C087E4898361E01C
:10405000CE0101960E94DB0B0E94590B83E08093F6
:1040600077056CE474E080E090E00E940329809181
:104070007705843079F58FE70E9477090E948A09D5
:10408000873441F520C061E070E08DE60E94DC1DC0
:1040900089E1E816F104F1F4D801EEEBF5E08D9139
:1040A000819385E0E73DF807D1F70E948E130BC09E
:1040B00061E070E08EE60E94DC1DF8018081809353
:1040C000D7050E942B0D81E006C061E070E08AEC0C
:1040D0000E94DC1D80E00E94BD1D0E94F91DA1967A
:1040E000E6E00C94272FA0E0B0E0E9E7F0E20C94C2
:1040F000092FCAECD3E014E606E035E0F32E44E0E5
:10410000E42E53E0D52E62E0C62E86EE95E00E94A6
:10411000E02B892B09F49BC086EE95E00E940D2CC4
:10412000282F809335044091340450E047305105E6
:1041300060F7FA01EE52FF4F0C94362F853B29F7BA
:1041400081E080933404E1CF823609F07DC0C092D3
:104150003404DBCF8093330480933204D092340450
:10416000D4CF9C01332730933104209330049091B5
:104170003204982790933204E0923404C6CF382F4B
:1041800022274091300450913104242B352B309359
:104190003104209330049091320498279093320494
:1041A000F09234042536310508F4AFCF61E070E0B9
:1041B0008CEC0E94DC1D81E00E94BD1D0E94F91D57
:1041C00043C020912E0430912F04F901E653FC4F97
:1041D000808390913204982790933204C90101960C
:1041E00090932F0480932E04209130043091310459
:1041F0008217930708F489CF0093340486CF809107
:10420000320482130BC060912E0470912F044AEC8B
:1042100053E0809133040E94001E0DC062E070E004
:104220008BEC0E94DC1D809133040E94BD1D8091A7
:104230006E050E94BD1DFE01812F11928A95E9F73E
:1042400010922F0410922E04109234045ECFCDB73A
:10425000DEB7E8E00C94252F81E080936F05809114
:104260006F05882349F086EE95E00E94E02B892BAC
:10427000B1F30E947320F3CF0895AAE2B0E0E3E423
:10428000F1E20C94072F0E94D4286B017C0181E09D
:104290000E947E0A86EE95E00E94E02B892B29F091
:1042A00086EE95E00E940D2CF5CF5E98409811E0C7
:1042B00072E6B72EE9E2AE2E03E00E94D4286C1914
:1042C0007D098E099F09693C710581059105E0F121
:1042D0001123D1F10E94D4286B017C015D9A419A8F
:1042E00080ED97E00E94A807B982EAE7F5E0DE01D9
:1042F00012968A2D01900D928A95E1F76AE2CE011D
:1043000001960E94DB0B5D98419880E090E00E944E
:10431000A807009377050E94590B62E370E080E0E4
:1043200090E00E94032980917705843061F4009326
:1043300077058FE70E9477090E948A0911E082348D
:1043400019F410E001C011E083E10E94F929892BE2
:10435000A1F411E012C05E9A409A5D9A419A86EEED
:1043600095E00E940D2C8D309105B9F06CF40A9700
:10437000A1F05E9840985D98419886EE95E00E9485
:10438000E02B892B41F799CF8332910579F0823464
:10439000910579F70E942C21ECCF62EB71E086EE5B
:1043A00095E00E94BA2A0E94931DE3CF0E941E1638
:1043B000E0CF8F929F92AF92BF92CF92DF92EF9217
:1043C000FF921F93CF93DF9383E10E94F929892BFA
:1043D00009F089C068EC70E080E090E00E94032959
:1043E00080E090E00E94A8070E94D4284B015C0165
:1043F0006B017C0180ECC80E82E1D81EE11CF11C2F
:104400000E94D4286C157D058E059F0530F483E14C
:104410000E94F929892BA1F364C083E10E94F92944
:10442000892B09F05EC080ED97E00E94A8070E94EA
:10443000D4286B017C01D0E0C1E088E4880E86E2DC
:10444000981EA11CB11C11E083E10E94F929892B5F
:1044500021F58C149D04AE04BF0430F480ED97E088
:104460000E94A807D1E0F0CF0E94D4286C197D09E2
:104470008E099F09693C71058105910528F30E9409
:10448000D4286B017C01C12719F080ED97E002C0B0
:1044900080E090E00E94A807D7CF80E090E00E94E3
:1044A000A807DD23B9F08091D70590E0019665E07B
:1044B00070E00E94AA2E8093D7050E942B0D0E94C7
:1044C000A9130E944A0D64EF71E080E090E00E9421
:1044D000032909C080E00E94DF060E94C2110E94E9
:1044E000410D0E943D21DF91CF911F91FF90EF90F0
:1044F000DF90CF90BF90AF909F908F900895CF9214
:10450000DF92EF92FF9280E00E94DA070E94B107EB
:1045100061E086E00E948D2961E085E00E948D299E
:1045200061E08EE00E948D2961E08FE00E948D297C
:1045300060E083E10E948D2960E088E00E948D297F
:1045400061E088E00E94C6290E949F0740E052EC8B
:1045500061E070E086EE95E00E94282D0E94A9138C
:104560000E944A0D0E948E138FEF8093AA040E942E
:10457000C60778940E94D4286B017C018091AA041C
:104580008F3F59F40E94D4286C197D098E099F0928
:10459000603D77408105910588F380ED97E00E94AA
:1045A000A80761E083E10E94C6295E9A409A86EEE0
:1045B00095E00E94E02B892B29F086EE95E00E9481
:1045C0000D2CF5CF6DEF72E086EE95E00E949B2AF0
:1045D00088E893E00E94300C64E173E086EE95E099
:1045E0000E949B2A4AE050E069E070E086EE95E088
:1045F0000E946B2B62E370E080E090E00E94032950
:1046000086EE95E00E94E02B04970CF186EE95E093
:104610000E940D2C82349105D1F486EE95E00E9423
:104620000D2C8E34910599F486EE95E00E940D2CA8
:104630008434910561F486EE95E00E940D2C8197FB
:1046400031F480E090E00E94A8070E943D21409153
:104650007B0550917C0560917D0570917E05DB01A5
:10466000CA010197A109B1090497A105B10590F408
:104670004093A904433051F42EE240EA56E861E049
:1046800070E086EE95E00E94A92D08C040E052EC53
:1046900061E070E086EE95E00E94282D0E94D9210D
:1046A0005E98409880E090E00E94A8070E948E13D8
:1046B0001092C9048091C30583FF11C080918F05BA
:1046C000882351F080919605882331F080919D05D3
:1046D000882311F087E001C085E08093C90480E061
:1046E0000E947E0A8091CA040E94B2090E94590B5E
:1046F00010923F0410923E0410923D04F12C8091E0
:10470000D8058F15B0F062E370E080E090E00E9481
:10471000032980ED97E00E94A80762E370E080E043
:1047200090E00E94032980E090E00E94A807F394A3
:10473000E6CF8091A20584FF08C0982F987181E090
:10474000983109F080E00E947E118FE00E94DA0724
:10475000FF90EF90DF90CF900895EF92FF920F932C
:104760001F93CF93DF938C016EE770E086EE95E0A8
:104770000E945906E801F12CF0E2EF2E8E018881AB
:104780008D57823048F46DE770E086EE95E00E9428
:10479000590688818E2588832196F801608186EEEE
:1047A00095E00E943A2CF394F9E0FF12E7CF6EE710
:1047B00070E086EE95E00E945906CDB7DEB7E6E0E0
:1047C0000C94272FA9E0B0E0E8EEF3E20C940F2F51
:1047D0009091CB0491110EC09EEF99838A836B83D5
:1047E00050E0559547954C832D83198618861F8276
:1047F0001E822EC04091D004842F90E0B4E09595A5
:104800008795BA95E1F7242F2F7030E08217930730
:1048100019F18DEF89831B82FE01349650E0842FBD
:1048200090E0A4E095958795AA95E1F7242F2F7045
:1048300030E08217930749F0DC01AF52BB4F8C91F7
:104840008193405F5F5F563051F74093D0045A83A5
:10485000CE0101960E94AD238091CB0490E0019699
:1048600066E070E00E94AA2E8093CB042996E2E0D5
:104870000C942B2FA0E0B0E0E0E4F4E20C94082FBD
:104880006C016EE770E086EE95E00E9459068601A5
:10489000E12CF12CC0E0D0E030E2B32EF8016081D1
:1048A00083E8860F823078F46DE770E086EE95E05D
:1048B0000E945906F80160816B2570E086EE95E054
:1048C0000E94590604C086EE95E00E943A2CE1143D
:1048D000F10459F0F80180819E01280F311DC901B2
:1048E000C92FDD27C80FD91FDD273FEFE31AF30AD1
:1048F00089E0E816F10459F028E0E216F10421F409
:104900008C2F8095F60180870F5F1F4FC7CFCDB7E3
:10491000DEB7E9E00C94242FA9E0B0E0E2E9F4E28C
:104920000C940F2FE82F362F8091CB0490E0019646
:1049300064E270E00E94AA2E8093CB0458E9598368
:1049400050E15A83813089F048F08230B9F08330E9
:10495000D9F48B8381EF8C833D8319C085E08B83F1
:1049600081EF8C832F5F2D8312C08B8381EF8C832B
:1049700084E6489FA00111245D8309C084E08B83F5
:1049800081EF8C83ED8303C00E94BB1104C0CE0174
:1049900001960E943A242996E2E00C942B2FA2E083
:1049A000B0E0E5EDF4E20C94042F182F762E2A8364
:1049B00049830E94E0286B017C018091E104809092
:1049C000CC049090CD04A090CE04B090CF042A8166
:1049D00049818823C1F0D701C60188199909AA091C
:1049E000BB094C015D0191EE89169EE29906A10476
:1049F000B10420F1241708F4422F202F672D812FB6
:104A00000E948C2413C0D701C60188199909AA09EC
:104A1000BB094C015D0191E3891695E79906A10454
:104A2000B10460F0672D812F0E94E223C092CC0474
:104A3000D092CD04E092CE04F092CF042296EDE025
:104A40000C94202FA2E2B0E0E8E2F5E20C94052FEE
:104A50008CE00E94990981110FC06CE173E086EE31
:104A600095E00E94CC2A5E9A409A80E00E947E0ADD
:104A70000E94590B5E98409886EE95E00E94E02BCC
:104A8000892B01F186EE95E00E940D2C9091A904EE
:104A9000992319F00E94BC13EFCF40913E0450E0DF
:104AA0009A012F5F3F4F2F71332760913F0470E0D1
:104AB0002617370709F3FA01E75BFB4F8083209342
:104AC0003E04DACF80917705843009F086C00E94D9
:104AD000E028611571058105910549F06093BB04DB
:104AE0007093BC048093BD049093BE040CC081E01D
:104AF00090E0A0E0B0E08093BB049093BC04A0934E
:104B0000BD04B093BE048091AD049091AE04816069
:104B10009093AE048093AD0483E0809377058FE794
:104B20000E94770909E614E00E948A09F80181933E
:104B30008F01F4E002371F07B9F7209172048091CA
:104B40006904982F922796FF3BC090E49227909398
:104B50007204982F98739833F1F410E0212F30E00D
:104B600080916904877090E0821793074CF11F5F72
:104B70002091A205812F90E0FC01E759FB4F24FF13
:104B800004C080810E949D11E9CF608186EE95E08E
:104B90000E943A2CE3CF8F7399F480916A0480933A
:104BA000B60480916B048093B40480916C0480936C
:104BB000B30480916F0490E09093AC048093AB04B5
:104BC00080913D04813019F482E080933D0480910E
:104BD0003D04833011F410923D040E94E0286B01E3
:104BE0007C018091AF049091B004A091B104B09188
:104BF000B2040097A105B105C9F0A7019601281BD1
:104C0000390B4A0B5B0BDA01C901883B9B40A105BC
:104C1000B10560F00E94C8098093B5041092AF04FA
:104C20001092B0041092B1041092B2048091BF04AB
:104C30009091C004A091C104B091C20446015701F3
:104C4000881A990AAA0ABB0A8AE795E00E94F40723
:104C500086169706A806B90608F4A9C0C092BF0434
:104C6000D092C004E092C104F092C2040E945706A0
:104C70008091AA048830A0F08091C3059091C4056A
:104C8000A091C505B091C6055CE1B695A79597952D
:104C900087955A95D1F7892B8A2B8B2B09F0AEC1BA
:104CA0008091AA048F5F8093AA048091BB049091A5
:104CB000BC04A091BD04B091BE040097A105B1054C
:104CC000F1F0C81AD90AEA0AFB0A8AE795E00E94BD
:104CD000F4076C157D058E059F0508F014C18091C1
:104CE000C30584FD04C080ED97E00E94A8071092E0
:104CF000BB041092BC041092BD041092BE049091AB
:104D00007204907C9093720450913E0480913F0411
:104D100020913D04581709F413C1223009F010C145
:104D2000905890937204E091A205E770F0E0E65885
:104D3000FC4F6081693008F0EBC0615040E04613E1
:104D4000E9C080933F0487E3840F90917204892B1C
:104D5000809372044093400483E080933D045D9A05
:104D6000419A809187059091C904911138C10E94A0
:104D7000790A8091CA040E94B209E091A205E77005
:104D8000F0E0E658FC4F608182E794E00E94940BCB
:104D9000E091CA04EF5FE093CA04E83109F42BC143
:104DA000F0E0E658FA4F8785882309F424C10E9471
:104DB000030C813069F58091A205887149F18091D9
:104DC000AD049091AE04880F991F9093AE04809328
:104DD000AD0483E0809377050E94590B0E94E02880
:104DE0006093AF047093B0048093B1049093B204C5
:104DF000672B682B692B61F481E090E0A0E0B0E0C4
:104E00008093AF049093B004A093B104B093B20424
:104E10008091A20584FF2BC08091BB049091BC04BB
:104E2000A091BD04B091BE04892B8A2B8B2BF9F085
:104E30008091AD049091AE048E7F0E942A09182FB4
:104E40006091AB048091B6040E94B213482F612F89
:104E50008091B50449A30E94B2130091D805282F70
:104E600049A16091B3048091B4040E94CF245D985D
:104E700041988091C7048130C1F018F08230B1F1BF
:104E8000CBC083E10E94F929892B09F0C5C081E0DC
:104E90008093C7040E94D4286093C3047093C40411
:104EA0008093C5049093C604B7C083E10E94F9299A
:104EB000892B31F50E94D428C090C304D090C4043B
:104EC000E090C504F090C6046C197D098E099F0915
:104ED000693E73408105910508F49EC082E080938D
:104EE000C70480ED97E00E94A80796C083E10E9466
:104EF000F929892B09F490C080E090E00E94A8076E
:104F00001092C70489C080E090E00E94A807F7CE05
:104F100068E014CF851709F414CF4F5F242F30E0D9
:104F200090E0F901EE58FB4FDC01A75BBB4F7C9191
:104F30007083F901E05CFB4F708301968F71FFCEA7
:104F40002430B1F42091400481E494E0A3E7B4E07C
:104F5000FC013E2F381B321718F431913D93F9CFE5
:104F600087E3820F90917204892B80937204F4CEB0
:104F70008091C704823059F49160909372045E9AD4
:104F8000409A8E010F5F1F4FF12CB80111C05E983F
:104F9000409880913D04811103C081E080933D04DD
:104FA00080913D04833069F784E080933D04E9CF2C
:104FB0008F2D69A37AA30E94DB15F8018193919349
:104FC0008F01F39469A17AA1F0E1FF12F1CF8091F2
:104FD000A20543E754E087700E947908C0CE882379
:104FE00009F4C5CE2091C80431E0320F3093C804D3
:104FF0002913BDCE0DC01092CA04D9CE8091AA0447
:10500000883011F45E9A409A89E08093AA04CFCE4A
:105010001092C8048150ABCEA296ECE00C94212FE4
:105020008230E8F4E82FF0E0EE0FFF1FE752FA4F6E
:1050300071836083813041F0809169008C7F842B83
:1050400080936900E89A089580916900440F551F84
:10505000440F551F837F842B80936900E99A08953C
:105060001F920F920FB60F9211242F933F934F93DD
:105070005F936F937F938F939F93AF93BF93EF93C0
:10508000FF938091D9059091DA05892B29F0E09161
:10509000D905F091DA050995FF91EF91BF91AF9194
:1050A0009F918F917F916F915F914F913F912F9140
:1050B0000F900FBE0F901F9018951F920F920FB672
:1050C0000F9211242F933F934F935F936F937F938E
:1050D0008F939F93AF93BF93EF93FF938091DB05E3
:1050E0009091DC05892B29F0E091DB05F091DC053E
:1050F0000995FF91EF91BF91AF919F918F917F9112
:105100006F915F914F913F912F910F900FBE0F9034
:105110001F9018951F920F920FB60F9211242F9384
:105120003F938F939F93AF93BF938091DE059091B0
:10513000DF05A091E005B091E1053091DD0523E0A8
:10514000230F2D3720F40196A11DB11D05C026E8BF
:10515000230F0296A11DB11D2093DD058093DE056E
:105160009093DF05A093E005B093E1058091E205FF
:105170009091E305A091E405B091E5050196A11D8C
:10518000B11D8093E2059093E305A093E405B093ED
:10519000E505BF91AF919F918F913F912F910F9016
:1051A0000FBE0F901F9018952FB7F8946091DE05F1
:1051B0007091DF058091E0059091E1052FBF089582
:1051C0003FB7F8948091E2059091E305A091E40542
:1051D000B091E50526B5A89B05C02F3F19F00196B3
:1051E000A11DB11D3FBF6627782F892F9A2F620F0F
:1051F000711D811D911D42E0660F771F881F991F49
:105200004A95D1F70895CF92DF92EF92FF92CF9314
:10521000DF936B017C010E94E028EB01C114D104F3
:10522000E104F10479F00E94E0286C1B7D0B683EDC
:105230007340A0F381E0C81AD108E108F108C85111
:10524000DC4FECCFDF91CF91FF90EF90DF90CF90CC
:105250000895789484B5826084BD84B5816084BDEE
:1052600085B5826085BD85B5816085BDEEE6F0E0DF
:10527000808181608083E1E8F0E01082808182603B
:105280008083808181608083E0E8F0E080818160BC
:105290008083E1EBF0E0808184608083E0EBF0E0EC
:1052A000808181608083EAE7F0E080818460808390
:1052B000808182608083808181608083808180683A
:1052C00080831092C1000895833081F028F48130EA
:1052D00099F08230A1F008958630A9F08730B9F0B6
:1052E0008430D1F4809180008F7D03C08091800054
:1052F0008F7780938000089584B58F7702C084B53E
:105300008F7D84BD08958091B0008F7703C0809118
:10531000B0008F7D8093B0000895CF93DF9390E02D
:10532000FC01ED50F44F2491FC01E95FF34F8491AF
:10533000882349F190E0880F991FFC01E15DF34F4C
:10534000A591B4918B5D934FFC01C591D4919FB70A
:10535000611108C0F8948C91209582238C938881E8
:1053600082230AC0623051F4F8948C91322F309528
:1053700083238C938881822B888304C0F8948C913A
:10538000822B8C939FBFDF91CF910895A1E0B0E075
:10539000ECECF9E20C940D2F282F30E0F901E152EA
:1053A000F44F8491F901ED50F44F1491F901E95F44
:1053B000F34F04910023C9F0882321F069830E94F0
:1053C00064296981E02FF0E0EE0FFF1FEB5DF34FE2
:1053D000A591B4919FB7F8948C91611103C0109579
:1053E000812301C0812B8C939FBF2196E4E00C9414
:1053F000292FCF93DF93282F30E0F901E152F44FAA
:105400008491F901ED50F44FD491F901E95FF34F24
:10541000C491CC2391F081110E946429EC2FF0E01B
:10542000EE0FFF1FE55EF34FA591B4912C912D2354
:1054300081E090E021F480E002C080E090E0DF9124
:10544000CF9108958E3008F08E50877020919D0185
:1054500090E4299F90011124822B80937C008091FD
:105460007A00806480937A0080917A0086FDFCCF78
:10547000809178002091790090E0922B0895A0E02F
:10548000B0E0E5E4FAE20C94092F6C017A01EB013B
:10549000E60EF71E00E010E0CE15DF0561F0699121
:1054A000D601ED91FC910190F081E02DC6010995A6
:1054B000080F191FF1CFC801CDB7DEB7E8E00C9493
:1054C000252F6115710589F0DB010D900020E9F7AA
:1054D000AD0141505109461B570BDC01ED91FC9188
:1054E0000280F381E02D0995089580E090E0089511
:1054F000EF92FF920F931F93CF93DF938C01FB01E9
:10550000C0E0D0E064917F018FEFE81AF80A6623CB
:1055100061F0D801ED91FC910190F081E02DC8017E
:105520000995C80FD91FF701EDCFCE01CDB7DEB772
:10553000E6E00C94272F0E94612A0895DC01ED918A
:10554000FC910190F081E02D099508950F931F9330
:10555000CF93DF93EC016DE00E949E2A8C016AE0FC
:10556000CE010E949E2A800F911FDF91CF911F9143
:105570000F9108950F931F93CF93DF93EC010E9437
:10558000782A8C01CE010E94A62A800F911FDF91FC
:10559000CF911F910F9108950F931F93CF93DF9396
:1055A000EC010E94612A8C01CE010E94A62A800F84
:1055B000911FDF91CF911F910F9108950F931F932A
:1055C000CF93DF93EC010E949E2A8C01CE010E94B2
:1055D000A62A800F911FDF91CF911F910F910895FF
:1055E000A1E2B0E0E6EFFAE20C94052F7C01C42EB4
:1055F000E52FCB01D22E19A221E02D1510F02AE0C3
:10560000D22E8E010F5D1F4F8D2C912CA12CB12C11
:105610006C2D7E2FA50194010E94BE2E8C2DD29E52
:1056200080191124015011098A3010F4805D01C0E5
:10563000895CF8018083211531054105510521F070
:10564000C22EE32FCA01E4CFB801C7010E94612A2C
:10565000A196ECE00C94212FA0E0B0E0E2E3FBE2A5
:105660000C94092FEC016A017B012115310541F4ED
:10567000E881F9810190F081E02D642F09951DC02A
:105680002A303105A9F477FF12C06DE20E949E2AEC
:105690008C0144275527BA014C195D096E097F0911
:1056A0002AE0CE010E94F02A800F911F06C02AE056
:1056B000B701A601CE010E94F02ACDB7DEB7E8E01F
:1056C0000C94252F9A01AB01662757FD6095762F24
:1056D0000E942C2B08950F931F93CF93DF93EC011F
:1056E0009A01AB01662757FD6095762F0E942C2BFF
:1056F0008C01CE010E94A62A800F911FDF91CF91CD
:105700001F910F9108952115310549F4DC01ED91A8
:10571000FC910190F081E02D642F099508950E947D
:10572000F02A08959A01462F50E060E070E00E9450
:10573000832B08959A01AB0160E070E00E94832BF7
:1057400008950F931F93CF93DF93EC010E94832B57
:105750008C01CE010E94A62A800F911FDF91CF916C
:105760001F910F9108950F931F93CF93DF93EC0137
:105770009A01AB0160E070E00E94832B8C01CE01A6
:105780000E94A62A800F911FDF91CF911F910F9148
:1057900008950F931F93CF93DF93EC019A01462F47
:1057A00050E060E070E00E94832B8C01CE010E94EB
:1057B000A62A800F911FDF91CF911F910F9108951D
:1057C000FC0124853585F901E05CFF4F80819181E2
:1057D000F901EE5BFF4F20813181821B930B8F73A8
:1057E00099270895FC0184859585FC01E05CFF4FB5
:1057F00040815181FC01EE5BFF4F208131814217D6
:10580000530741F00190F081E02DE80FF91F8081EE
:1058100090E008958FEF9FEF0895FC0184859585B2
:10582000FC01E05CFF4F40815181FC01EE5BFF4FCA
:10583000208131814217530779F0A081B181A80FEF
:10584000B91F8C91208131812F5F3F4F2F733327F8
:105850003183208390E008958FEF9FEF0895FC013E
:1058600081A1882329F0A489B5898C9186FFFBCF7B
:1058700011A20895CF93DF93FC0126853785D901C6
:10588000A05CBF4F8D919C91119701968F739927C2
:10589000E901CE5BDF4F4881598184179507D9F321
:1058A0000D90BC91A02DA20FB31F6C93A685B78558
:1058B000A05CBF4F11969C938E93A689B7892C91BB
:1058C00081E090E0078C02C0880F991F0A94E2F7EC
:1058D000282B2C9381E081A30488F589E02D808119
:1058E0008064808381E090E0DF91CF9108950895F6
:1058F0001F920F920FB60F9211242F933F934F9345
:105900008F939F93EF93FF938091C00082FD1CC003
:105910004091C60080918C0690918D0601968F7300
:10592000992720918E0630918F068217930771F088
:10593000E0918C06F0918D06E45BF94F40839093E3
:105940008D0680938C0602C08091C600FF91EF9176
:105950009F918F914F913F912F910F900FBE0F907C
:105960001F90189586EE95E00E94E02B892B11F090
:105970000E94772C08951F920F920FB60F92112458
:105980002F933F938F939F93EF93FF93209148061C
:105990003091490680914A0690914B0628173907A5
:1059A00031F48091C1008F7D8093C10014C0E091DB
:1059B0004A06F0914B06E85FF94F208180914A0634
:1059C00090914B0601968F73992790934B06809385
:1059D0004A062093C600FF91EF919F918F913F91CE
:1059E0002F910F900FBE0F901F901895A0E0B0E080
:1059F000ECEFFCE20C94052FFC011382128288EE7E
:105A000093E0A0E0B0E084839583A683B7838CEB1A
:105A100093E0918380837587648757874687318BAE
:105A2000208B138B028BF58AE48AD78AC68AB18EC3
:105A3000A08E938E828E8F85848F8889858F8989A9
:105A4000868F8A89878F8B8980A3ECE00C94212F25
:105A5000CF92DF92EF92FF92CF93DF93EC016A0136
:105A60007B01411581EE580761057105F9F0EC895C
:105A7000FD8981E090E008A002C0880F991F0A9478
:105A8000E2F7808360E079E08DE390E0A701960182
:105A90000E94BE2E21503109410951095695479562
:105AA00037952795211580E1380798F0EC89FD8915
:105AB000108260E874E88EE190E0A70196010E94F0
:105AC000BE2E215031094109510956954795379508
:105AD0002795E889F9893083EA89FB89208319A20F
:105AE000EE89FF89408181E090E09C010C8C02C02E
:105AF000220F331F0A94E2F7422B4083EE89FF897D
:105B000040819C010D8C02C0220F331F0A94E2F7E2
:105B1000422B4083EE89FF8940819C010E8C02C09C
:105B2000220F331F0A94E2F7422B4083EE89FF894C
:105B300020810F8C02C0880F991F0A94E2F780958C
:105B400082238083DF91CF91FF90EF90DF90CF9001
:105B50000895BF92CF92DF92EF92FF92CF93DF939F
:105B6000EC016A017B01B22E411581EE58076105F7
:105B70007105F9F0EC89FD8981E090E008A002C090
:105B8000880F991F0A94E2F7808360E079E08DE343
:105B900090E0A70196010E94BE2E215031094109D3
:105BA00051095695479537952795211580E1380776
:105BB00098F0EC89FD89108260E874E88EE190E04D
:105BC000A70196010E94BE2E2150310941095109B9
:105BD0005695479537952795E889F9893083EA895D
:105BE000FB892083E88DF98DB082EE89FF894081A1
:105BF00081E090E09C010C8C02C0220F331F0A94BC
:105C0000E2F7422B4083EE89FF8940819C010D8C95
:105C100002C0220F331F0A94E2F7422B4083EE8921
:105C2000FF8940819C010E8C02C0220F331F0A9411
:105C3000E2F7422B4083EE89FF8920810F8C02C05E
:105C4000880F991F0A94E2F7809582238083DF9161
:105C5000CF91FF90EF90DF90CF90BF9008958F92FB
:105C60009F92AF92BF92CF92DF92EF92FF920F93EB
:105C70001F9381E08F9385E08F9387E08F9383E07C
:105C80008F9384E08F93E6EC8E2E912CF2ECAF2E66
:105C9000B12CA1ECCA2ED12CB0ECEB2EF12C04ECE3
:105CA00010E025EC30E048E056E06CE476E086EE6B
:105CB00095E00E94F62C0F900F900F900F900F9090
:105CC0001F910F91FF90EF90DF90CF90BF90AF901A
:105CD0009F908F9008950E9429290E947F22C2EBF5
:105CE000DCE20E9422252097E1F30E94B22CF9CF3A
:105CF000A29FB001B39FC001A39F700D811D11240D
:105D0000911DB29F700D811D1124911D08950E9457
:105D1000782EA59F900DB49F900DA49F800D911D8E
:105D200011240895B7FF0C94872E0E94872E821BA2
:105D3000930B0895DB018F939F930E94872EBF9151
:105D4000AF91A29F800D911DA39F900DB29F900DCA
:105D50001124089597FB072E16F4009407D077FDC1
:105D600009D00E943C2F07FC05D03EF49095819508
:105D70009F4F0895709561957F4F0895A1E21A2E67
:105D8000AA1BBB1BFD010DC0AA1FBB1FEE1FFF1FDF
:105D9000A217B307E407F50720F0A21BB30BE40B2F
:105DA000F50B661F771F881F991F1A9469F7609576
:105DB0007095809590959B01AC01BD01CF01089530
:105DC000052E97FB1EF400940E94F72E57FD07D076
:105DD0000E94BE2E07FC03D04EF40C94F72E509573
:105DE0004095309521953F4F4F4F5F4F08959095C7
:105DF0008095709561957F4F8F4F9F4F08952F929B
:105E00003F924F925F926F927F928F929F92AF924A
:105E1000BF92CF92DF92EF92FF920F931F93CF9397
:105E2000DF93CDB7DEB7CA1BDB0B0FB6F894DEBF2E
:105E30000FBECDBF09942A88398848885F846E8454
:105E40007D848C849B84AA84B984C884DF80EE809E
:105E5000FD800C811B81AA81B981CE0FD11D0FB6A7
:105E6000F894DEBF0FBECDBFED010895EE0FFF1F0A
:105E70000590F491E02D0994AA1BBB1B51E107C0CA
:105E8000AA1FBB1FA617B70710F0A61BB70B881FCA
:105E9000991F5A95A9F780959095BC01CD01089559
:105EA0008F929F92AF92BF92CF92DF92EF92FF922A
:105EB000CF93DF93EC01688179818A819B816115A1
:105EC00071058105910521F464E279ED8BE597E098
:105ED0002DE133EF41E050E00E94E02E49015A01EC
:105EE0009B01AC01A7EAB1E40E94872E6B017C0103
:105EF000ACEEB4EFA50194010E94952EC60ED71EFC
:105F0000E81EF91EF7FE06C081E0C81AD108E108B4
:105F100080E8F80AC882D982EA82FB82C701B6010A
:105F20009F77DF91CF91FF90EF90DF90CF90BF9060
:105F3000AF909F908F9008950E94502F089586E013
:105F400091E00E94502F089560930601709307011D
:105F5000809308019093090108952F923F925F92D8
:105F60006F927F928F929F92AF92BF92CF92DF9269
:105F7000EF92FF920F931F93CF93DF938B01EA0170
:105F80006115710521F0DB018C9311969C9320978C
:105F900039F09E01225031092332310508F0D8C072
:105FA0007C016701BFEFCB1ADB0A5601F701608065
:105FB000862D90E00E94DF30892B11F07601F1CF21
:105FC000FDE26F120AC0570182E0A80EB11CD70192
:105FD00011966C90772473940BC0BBE26B1207C0D0
:105FE0005701E2E0AE0EB11CD70111966C90712CF6
:105FF000CE018F7E892B89F4B0E36B1237C0F50197
:1060000080818F7D8835D1F46180F2E0AF0EB11CC4
:10601000872D8260782EC0E1D0E0CA30D10551F1E1
:10602000C031D10521F0C830D10599F409C0CC2484
:10603000CA94DC2CEC2CAFE0FA2E22C0209769F732
:10604000C8E0D0E0CC24CA94DC2CEC2CFFE1FF2E7D
:1060500017C06FEF7FEFCB019E01442737FD4095BE
:10606000542F0E94BE2E69017A010AC02097A9F61A
:10607000CAE0D0E0E9E9CE2EDC2CEC2CE9E1FE2EE2
:10608000F50160E020E030E0A9014E01AA2497FC70
:10609000A094BA2C1F0170ED572E560CA9E0A5153F
:1060A00070F48FEB860D8A3118F499EC592E06C0E6
:1060B0008FE9860D8A3148F589EA582E560C852DD0
:1060C00090E08C179D070CF56F3FD9F0C216D306F0
:1060D000E406F50698F0C501B4010E949A2E9B01D2
:1060E000AC01852D90E0A0E0B0E0280F391F4A1FD9
:1060F0005B1F281739074A075B0710F46FEF01C0D1
:1061000061E03196D1016C90C5CF0115110551F0B8
:10611000662311F0319703C071FE04C03297D80195
:10612000ED93FC9370FE07C05095409530952195F6
:106130003F4F4F4F5F4F67FF10C082E290E0909358
:106140009106809390066FEF7FEF8FEF9FEF07C070
:1061500060E070E080E090E002C0B901CA01DF9128
:10616000CF911F910F91FF90EF90DF90CF90BF9054
:10617000AF909F908F907F906F905F903F902F9007
:106180000895FC0188279927E89421912032E9F3AA
:10619000293010F02E30C8F32B3241F02D3239F473
:1061A000689404C00E941331820F911D21912053E5
:1061B0002A30C0F31EF4909581959F4F0895911158
:1061C00050C0803219F089508550D0F7089548ECBE
:1061D00053E00E94EC300895FA01A191B08100973C
:1061E00019F41097E1F0CD01DC01CD010D900020F4
:1061F00011F4C00113C0FB012191222319F02015D5
:10620000D9F7F3CFFB012191201519F41E921196B5
:1062100006C02223C1F70D900020A1F7D001FA019A
:10622000A193B08308957AE0979F902D879F802D4A
:10623000910D11240895F999FECF92BD81BDF89A70
:10624000992780B50895262FF999FECF1FBA92BDE0
:1062500081BD20BD0FB6F894FA9AF99A0FBE019647
:0C6260000895992788270895F894FFCF2F
:10626C0000009206200001000000FF000200020066
:10627C000200020002000200020002000200020002
:10628C00020002000200020002000280250000054C
:10629C00400AA1204EA50020244EA52C2330C0126C
:1062AC0000001A400AA1204EA5001B1E27522C23C9
:1062BC00308025000005400AA1204EA50020244E68
:1062CC00A52C2330004B000006400AD0009D49004D
:1062DC007B289D492C233000E1000005400A450134
:1062EC00D7DC03B81E0EBF00232E48E801008A40FD
:1062FC000A6001555502AD1E20000023C8015458F8
:10630C002074696D656F75742100596573004E6F4B
:10631C00002C00386368004E2F41002C205B005D80
:10632C002028002900486F70206368616E6E656CD0
:10633C00200020402000456E746572696E672061F4
:10634C0064617074697665206368616E6E656C203B
:10635C0073656C656374696F6E2C207069636B690F
:10636C006E673A007363616E6E6572206D6F646563
:10637C00004E4F5420454E41424C45440053656EEF
:10638C0064696E672073657474696E677320746FCB
:10639C002052580A00526573657474696E672073D5
:1063AC00657474696E6773206F6E2052580A0041D1
:1063BC00626F727465642065646974730A00696E37
:1063CC0076616C69642073656C656374696F6E00CB
:1063DC000D0A496E76616C696420696E7075742063
:1063EC002D206469736361726465642107005365D1
:1063FC007474696E677320736176656420746F20A2
:10640C00454550524F4D0A0052657665727465646D
:10641C002073657474696E67732066726F6D2045A6
:10642C004550524F4D0A004C6F61646564206661A3
:10643C0063746F72792064656661756C74730A009D
:10644C004B657920616E64206368616E6E656C7358
:10645C002072616E646F6D697A65640A004F7065B5
:10646C006E4C52536E672054582073746172746969
:10647C006E672000206F6E20485720006D6F64758A
:10648C006C65206C6F636B65643F00342B34003893
:10649C0000382B340031320031322B3400313600CD
:1064AC0050504D0052535349005344410053434CF8
:1064BC0000525844005458440041494E004C424547
:1064CC0045500053504B54524D00534255530053BA
:1064DC00554D44004C4C494E440000070B0C101118
:1064EC001500B7012B032F033103350338033D038C
:1064FC00B7014003440349034D03510355035903AA
:10650C005D0363036A036F0374038D028D028D02B6
:10651C008D02160A13223129000000003A2C3F2A62
:08652C00E02B0D2CF22B2F2CAB
:107E00000F92CDB7DEB7112484B714BE81FFF1D035
:107E100082E08093C00088E18093C10086E0809377
:107E2000C20080E18093C4008EE0CDD088249924E4
:107E3000CC24C394F5E0DF2EE1E1EE2E73E0F72EC3
:107E4000B6D0082F813479F4B2D08983C2D0898129
:107E5000823811F481E005C0813811F485E001C059
:107E600083E09ED09AC0823411F484E103C085344B
:107E700019F485E0B6D091C0853561F498D0082F0B
:107E800010E095D090E0982E8824802A912A880CC2
:107E9000991C82C0863521F484E0A3D080E0E1CF34
:107EA000843609F04CC083D082D0A82E80D0B82E62
:107EB00000E011E07CD0F80181938F01AE16D1F77C
:107EC00088D0FB2DF53489F4E0E0F1E00BC0F9999E
:107ED000FECF92BC81BC0894811C911C819180BD15
:107EE000FA9AF99AEA1598F358C08B2D863409F05E
:107EF00054C0F401F7BEE89507B600FCFDCFF401CD
:107F0000A0E0B1E02C9130E011968C91119790E0B7
:107F1000982F8827822B932B12960C01C7BEE895C9
:107F20001124329681E0A038B80761F7F401D7BE7A
:107F3000E89507B600FCFDCFE7BEE8952EC0843774
:107F4000F1F435D034D0182F32D0B82E42D0FB2DDA
:107F5000F63421F4F40105914F010CC0FB2DF534EA
:107F600049F4F999FECF92BC81BC0894811C911C04
:107F7000F89A00B5802F14D0115049F70EC08537FC
:107F800039F427D08EE10CD085E90AD08FE069CF93
:107F9000813511F488E017D01CD080E101D050CF9A
:107FA0009091C00095FFFCCF8093C600089580910A
:107FB000C00087FFFCCF8091C00084FD01C0A89560
:107FC0008091C6000895E0E6F0E098E19083808318
:107FD0000895EDDF803219F088E0F5DFFFCF84E10E
:107FE000DFCF1F93182FE3DF1150E9F7F2DF1F9166
:0E7FF0000895282E80E0E7DFEE27FF27099492
:027FFE0001057B
:0400000300007E007B
:00000001FF
